:020000040000FA
:1000000005EF33F012001200B3EF01F0120001000F
:1000100076660000E0070000650100000F0E9316F1
:100020008116939493968194819600D90F0E811630
:10003000300E811227D81FD90F0E8116300E811273
:1000400021D819D90F0E8116300E81121BD813D961
:100050000F0E8116818A16D8280EE66E17D8E55243
:10006000080EE66E13D8E552010EE66E0FD8E55283
:10007000060EE66E0BD8E5520C0EE66E07D8E5527A
:1000800000D0120081861CD981961200D9CFE6FFDC
:10009000E1CFD9FF1AD9819481960F0E8116FE0EF9
:1000A000DB50F00B8112EEDF0F0E8116FE0EDB38F7
:1000B000F00BF00B8112E6DF00D0E552E7CFD9FF5D
:1000C0001200D9CFE6FFE1CFD9FFFFD88184819616
:1000D0000F0E8116FE0EDB50F00B81128186F0D8D8
:1000E00081960F0E8116FE0EDB38F00BF00B81129D
:1000F0008186E6D8819600D0E552E7CFD9FF12007D
:10010000D9CFE6FFE1CFD9FFFD0EDBCFF6FFFE0E24
:10011000DBCFF7FF0800F55011E0FD0EDBCFF6FF57
:10012000FE0EDBCFF7FF0800F550E66ECADFE552A2
:10013000FD0EDB2AFE0E01E3DB2AE6D700D0E552F6
:10014000E7CFD9FF1200D9CFE6FFE1CFD9FFFD0EEF
:10015000DBCFE9FFFE0EDBCFEAFFEF5010E0FD0E34
:10016000DBCFE9FFFE0EDBCFEAFFEF50E66EA9DF43
:10017000E552FD0EDB2AFE0E01E3DB2AE8D700D0B4
:10018000E552E7CFD9FF1200D9CFE6FFE1CFD9FF83
:10019000E652FE0EDB0404E1FD0EDB50800FDF6E45
:1001A000FE0EDB50020804E1FD0EDB50C00FDF6ED7
:1001B000DFCFE6FF6BDFE552E552E552E7CFD9FF2F
:1001C0001200D9CFE6FFE1CFD9FF020EE126E66AA1
:1001D000FE0EDBCFE6FFD8DFE552E552DE6ADD6AD0
:1001E000DECF14F0DDCF15F0D890155004E6100ED8
:1001F000145C000E155809E2200EE66E62DFE5522F
:10020000DF2A010E01E3DB2AEBD7E66AFE0EDBCF25
:10021000E6FFBADFE552E552020EE15C02E2E16A76
:10022000E552E16EE552E7CFD9FF1200D9CFE6FFE4
:10023000E1CFD9FF020EE126DE6ADD6ADECF14F0DF
:10024000DDCF15F0D890155004E6100E145C270E83
:10025000155806E20000DF2A010E01E3DB2AEED783
:1002600000D0020EE15C02E2E16AE552E16EE55285
:10027000E7CFD9FF1200D9CFE6FFE1CFD9FF020EB9
:10028000E126DE6ADD6ADECF14F0DDCF15F0D8900E
:10029000155004E6C40E145C090E155806E2000061
:1002A000DF2A010E01E3DB2AEED700D0020EE15C6B
:1002B00002E2E16AE552E16EE552E7CFD9FF1200B2
:1002C00000000000000000001200D9CFE6FFE1CFDF
:1002D000D9FF020EE126DE6ADD6ADECF14F0DDCF43
:1002E00015F0D890155004E6E80E145C030E15586E
:1002F00006E20000DF2A010E01E3DB2AEED700D080
:10030000020EE15C02E2E16AE552E16EE552E7CFFE
:10031000D9FF1200D9CFE6FFE1CFD9FF81940F0EAC
:100320008116FE0EDB504009F00B8112C9DFAADEF8
:100330000F0E8116FE0EDB38F00BF00B8112C0DFC2
:10034000A1DE00D0E552E7CFD9FF12000000000087
:10035000000000000000000000000000000000009D
:10036000000000001200DACFE4FFE2CFDAFFE9CFAD
:10037000E4FFEACFE4FFF6CFE4FFF7CFE4FFF5CFE9
:10038000E4FFF3CFE4FFF4CFE4FFFACFE4FF00EEA5
:1003900000F0140EE80403E3EECFE4FFFBD700EE19
:1003A00014F0140EE80403E3EECFE4FFFBD7E652AB
:1003B0009D50200B30E09E50200B2DE05FEC32F082
:1003C0000701116FABA407D0AB9EC5810F2B000EA8
:1003D0001023AB8E01D0C591ABA207D0AB98C583DB
:1003E000AB880D2B000E0E2301D0C593ACA2FED717
:1003F000070104C7E9FF05C7EAFF042B000E052328
:1004000011C7EFFFA00E045D000E055904E3600E56
:10041000046F000E056F9D50010B1CE09E50010BF8
:1004200019E00701C62B000EC723140EC65D000E8F
:10043000C75907E3C66BC76BC585CA2B000ECB2314
:100440008978DB0EE66E0B0EE66E7EEC32F0E5523E
:10045000E5529E90F250100B1CE0F250020B19E096
:10046000070111510CE11B0E116F9D9A9E9A600EAF
:10047000046F000E056F04C702F705C703F7F29279
:10048000F2989D9A010ECC6FCD6B400EE66E9CDB10
:10049000E552A050400B1EE0A150400B1BE077AE90
:1004A00004D0010E0701926F936BA09CA19C0701E1
:1004B0001B0E116F440EE66E87DBE5520A0EE66EE8
:1004C00083DBE5520D0EE66E7FDBE55281A202D0A2
:1004D000A1EC18F0A050200B1EE0A150200B1BE057
:1004E00077AC04D0010E0701946F956BA09AA19A86
:1004F00007011B0E116F470EE66E66DBE5520A0E12
:10050000E66E62DBE5520D0EE66E5EDBE55281A221
:1005100002D0A1EC18F0E55200EE27F0140EE8042A
:1005200003E3E5CFEDFFFBD700EE13F0140EE80474
:1005300003E3E5CFEDFFFBD7E5CFFAFFE5CFF4FF0F
:10054000E5CFF3FFE5CFF5FFE5CFF7FFE5CFF6FF0A
:10055000E5CFEAFFE5CFE9FFE5CFDAFF1100D9CF1C
:10056000E6FFE1CFD9FF020EE126829A100EDE6E81
:10057000DD6ADECF14F0DDCF15F0153404E214503F
:100580000008000E15543EE2FE0EDB50800B02E127
:10059000829801D08288640EE66EE66AE66AE66AB0
:1005A0001FEC0DF0E552E552E552E5528286640EED
:1005B000E66EE66AE66AE66A1FEC0DF0E552E55281
:1005C000E552E5528296640EE66EE66AE66AE66AEF
:1005D0001FEC0DF0E552E552E552E552FD0EDBCF82
:1005E00014F0FE0EDBCF15F0D89014361536FD0E44
:1005F00014C0DBFFFE0E15C0DBFFDF06010E01E2BB
:10060000DB06B7D7828A020EE15C02E2E16AE552BC
:10061000E16EE552E7CFD9FF1200E66AD00EE66E32
:100620009EDFE552E552200EE66E4E0EE66EE66A5D
:10063000E66A1FEC0DF0E552E552E552E55207017E
:10064000A20EC06FEE0EC16F030EC26FC36BA20E7F
:10065000E66E300EE66E83DFE552E552EE0EE66E94
:10066000210EE66E7CDFE552E552030EE66E320E99
:10067000E66E75DFE552E552E66A230EE66E6FDF41
:10068000E552E552100EE66E270EE66EE66AE66A61
:100690001FEC0DF0E552E552E552E552E66A900E88
:1006A000E66E5DDFE552E552E66AC00EE66E57DFA4
:1006B000E552E552100EE66E270EE66EE66AE66A31
:1006C0001FEC0DF0E552E552E552E552E66A500E98
:1006D000E66E45DFE552E552100EE66E270EE66E39
:1006E000E66AE66A1FEC0DF0E552E552E552E55286
:1006F0001200D9CFE6FFE1CFD9FFE66AD00EE66E51
:100700002EDFE552E552100EE66E270EE66EE66A23
:10071000E66A1FEC0DF0E552E552E552E552FB0E9C
:10072000DBCF14F0FC0EDBCF15F0FD0EDBCF16F0A7
:10073000FE0EDBCF17F07CC70CF07DC70DF07EC737
:100740000EF07FC70FF014C007F015C008F016C0F8
:1007500009F017C00AF031EC27F01AEC28F006C0B7
:10076000C0F707C0C1F708C0C2F709C0C3F7D95026
:10077000F90FE96EFF0EDA20EA6E000ED880EE5413
:10078000000EED5439E20701C051156A000F146ED6
:10079000340E152214C0E6FF15C0E6FFE0DEE55278
:1007A000E5520701C151156A000F146E250E15227E
:1007B00014C0E6FF15C0E6FFD2DEE552E5520701A0
:1007C000C251156A000F146E360E152214C0E6FFD2
:1007D00015C0E6FFC4DEE552E5520701C351156AB4
:1007E000000F146E270E152214C0E6FF15C0E6FF99
:1007F000B6DEE552E55238D00701C051156A000F48
:10080000146E300E152214C0E6FF15C0E6FFA7DEF9
:10081000E552E5520701C151156A000F146E210E11
:10082000152214C0E6FF15C0E6FF99DEE552E55239
:100830000701C251156A000F146E320E152214C042
:10084000E6FF15C0E6FF8BDEE552E5520701C35116
:10085000156A000F146E230E152214C0E6FF15C092
:10086000E6FF7DDEE552E552100EE66E270EE66EDF
:10087000E66AE66A1FEC0DF0E552E552E552E552F4
:10088000E66A900EE66E6BDEE552E552E66AC00E51
:10089000E66E65DEE552E552100EE66E270EE66E58
:1008A000E66AE66A1FEC0DF0E552E552E552E552C4
:1008B000E66A500EE66E53DEE552E552100EE66E25
:1008C000270EE66EE66AE66A1FEC0DF0E552E55289
:1008D000E552E552E552E7CFD9FF1200D9CFE6FF46
:1008E000E1CFD9FF040EE126D9CFE9FFDACFEAFF45
:1008F000FB0EDBCFEEFFFC0EDBCFEEFFFD0EDBCF02
:10090000EEFFFE0EDBCFEEFFD60EE66E080EE66EB5
:10091000D9CFE9FFDACFEAFFEECFE6FFEECFE6FF71
:10092000EECFE6FFEFCFE6FF07EC2EF0146E060EDB
:10093000E15E1450D60EE66E080EE66E0ED9E55254
:10094000E552F3CF16F7F4CF17F7090EE66E3CD950
:10095000E552D9CFE9FFDACFEAFFEECF14F0EECFC0
:1009600015F0EECF16F0EFCF17F01450E66EC7EC8F
:100970000CF0E552090EE66E27D9E552D9CFE9FF12
:10098000DACFEAFFEECF14F0EECF15F0EECF16F08F
:10099000EFCF17F0080ED8901732163215321432F6
:1009A000E806F9E114C0DFFF010E15C0DBFF020EFF
:1009B00016C0DBFF030E17C0DBFFD9CFE9FFDACF8C
:1009C000EAFFEECF14F0EECF15F0EECF16F0EFCF3A
:1009D00017F01450E66EC7EC0CF0E552090EE66E07
:1009E000F3D8E552000EDFCFE6FFC7EC0CF0E5527E
:1009F000090EE66EE9D8E552D9CFE9FFDACFEAFF72
:100A0000EECF14F0EECF15F0EECF16F0EFCF17F0DB
:100A1000080ED8901732163215321432E806F9E172
:100A200014C0DFFF010E15C0DBFF020E16C0DBFF96
:100A3000030E17C0DBFFD9CFE9FFDACFEAFFEECF15
:100A400014F0EECF15F0EECF16F0EFCF17F01450F4
:100A5000E66EC7EC0CF0E552090EE66EB5D8E5522D
:100A6000D9CFE9FFDACFEAFFEECF14F0EECF15F0E1
:100A7000EECF16F0EFCF17F0080ED89017321632DF
:100A800015321432E806F9E114C0DFFF010E15C07B
:100A9000DBFF020E16C0DBFF030E17C0DBFF000EEC
:100AA000DFCFE6FFC7EC0CF0E552090EE66E8CD8FE
:100AB000E5529AD8040EE15C02E2E16AE552E16E89
:100AC000E552E7CFD9FF1200400EE66EE66A740EDB
:100AD000E66EFFEC31F0E552E552E5529F8AD08E8A
:100AE0009D9AF29CF29E1200D9CFE6FFE1CFD9FF8A
:100AF000020EE126DE6ADD6AFD0EDBCFF6FFFE0E9A
:100B0000DBCFF7FF0800F55015E0FD0EDBCFF6FF59
:100B1000FE0EDBCFF7FF0800F550E66E55D8E55224
:100B2000DF2A010E01E3DB2AFD0EDB2AFE0E01E3C4
:100B3000DB2AE2D7DECF14F0DDCF15F014C0F3FFCF
:100B400015C0F4FF020EE15C03E200D0E16AE55259
:100B5000E16EE552E7CFD9FF1200D9CFE6FFE1CF32
:100B6000D9FF020EE126DE6ADD6AFD0EDBCFE9FF6A
:100B7000FE0EDBCFEAFFEF5014E0FD0EDBCFE9FF06
:100B8000FE0EDBCFEAFFEF50E66E1ED8E552DF2AFD
:100B9000010E01E3DB2AFD0EDB2AFE0E01E3DB2A58
:100BA000E4D7DECF14F0DDCF15F014C0F3FF15C08D
:100BB000F4FF020EE15C03E200D0E16AE552E16E6F
:100BC000E552E7CFD9FF1200D9CFE6FFE1CFD9FF39
:100BD000ACA2FED7FE0EDBCFE6FFB6EC32F0E5525C
:100BE000E552E7CFD9FF12000D0EE66EEDDFE552BC
:100BF0000A0EE66EE9DFE5521200D9CFE6FFE1CF3B
:100C0000D9FFE65207010451021902E10551031907
:100C100001E1F8D702C7E9FF03C7EAFF022B000E84
:100C20000323EFCFDFFFA00E025D000E035904E3A4
:100C3000600E026F000E036FDF5000D0E552E552E8
:100C4000E7CFD9FF1200D9CFE6FFE1CFD9FFFF0EE2
:100C5000E76EFD0EDBCF14F0FE0EDBCF15F0E75094
:100C60001416156A1450A96EFD0EDBCF14F0FE0E9B
:100C7000DBCF15F015C014F0156A030E1414AA6E1C
:100C8000A69EA69CA680E80EE66E030EE66EE66AB9
:100C9000E66A1FEC0DF0E552E552E552E552A85028
:100CA00000D0E552E7CFD9FF1200D9CFE6FFE1CF60
:100CB000D9FF020EE1260701C4AF11D0E76EFD0E89
:100CC000DBCF14F0FE0EDBCF15F0E7501426000E3C
:100CD0001522FD0E14C0DBFFFE0E15C0DBFFFD0E5E
:100CE000DBCF14F0FE0EDBCF15F015C014F0156A43
:100CF000030E1414AA6EFF0EE76EFD0EDBCF14F088
:100D0000FE0EDBCF15F0E7501416156A1450A96ECD
:100D1000FC0EDB50A86EA69EA684A69CF2AE04D064
:100D2000F29E010EDE6EDD6A550EA76EAA0EA76E4C
:100D3000A682A1A8FED7A198A694D9CFE9FFDACFC1
:100D4000EAFF010EEE1801E1ED5001E1F28E020E14
:100D5000E15C02E2E16AE552E16EE552E7CFD9FFDC
:100D60001200D9CFE6FFE1CFD9FFFB0EDBCFE9FFC1
:100D7000FC0EDBCFEAFFEF5022E0FB0EDBCFE9FFFA
:100D8000DB2AFC0EDBCFEAFF01E3DB2AEF50E66E45
:100D9000D950FD0FE96EFF0EDA20EA6EEECF14F0A7
:100DA000EDCF15F0020EEE26000EEF2214C0E6FF86
:100DB00015C0E6FF7ADFE552E552E552D6D7E55297
:100DC000E7CFD9FF1200D9CFE6FFE1CFD9FF040E5C
:100DD000E1260701C4AF17D0FD0EDBCF14F0FE0EE5
:100DE000DBCF15F0040ED89014361536E804FBE17D
:100DF000000E1426020E1522FD0E14C0DBFFFE0E9F
:100E000015C0DBFF12D0FD0EDBCF14F0FE0EDBCFE2
:100E100015F0050ED89014361536E804FBE1FD0EEA
:100E200014C0DBFFFE0E15C0DBFF020EDB6A030EF3
:100E3000DB6AD950FD0FE96EFF0EDA20EA6EFF0E75
:100E4000D880EE54030EED5401E242D0FD0EDBCF0C
:100E5000E6FFFE0EDBCFE6FFF6DEE552E552DE6E84
:100E6000DD6AD9CFE9FFDACFEAFFEE50ED1001E1FC
:100E70002FD00701C451800B0EE0020EDBCF14F01F
:100E8000030EDBCF15F0153404E214500F08000EEA
:100E9000155401E21DD0C4BF05D0DFCFE6FF94DEBC
:100EA000E55205D0DFCFE6FF61EC00F0E552FD0E24
:100EB000DB2AFE0E01E3DB2A020EDB2A030E01E32E
:100EC000DB2AD9CFE9FFDACFEAFFEE50ED10B1E12E
:100ED000E80EE66E030EE66EE66AE66A1FEC0DF0BB
:100EE000E552E552E552E552040EE15C02E2E16AA8
:100EF000E552E16EE552E7CFD9FF1200D9CFE6FF08
:100F0000E1CFD9FF0A0EE1260701280E006F090E76
:100F1000016FFC0EDB50010801E2E0D0FC0EDB505B
:100F200028E1FD0EDBCF14F0FE0EDBCF15F0060E30
:100F300014C0DBFF070E15C0DBFF080EDB6A090ECD
:100F4000DB6A00C7E6FF01C7E6FFD950060FE96E6E
:100F5000DACFEAFFEECFE6FFEECFE6FFEECFE6FF19
:100F6000EFCFE6FF07EC2EF0146E060EE15E145094
:100F700010D000C7E6FF01C7E6FFFD0EDBCFE6FF9E
:100F8000FE0EDBCFE6FF6DEC2DF0E552E552E552AB
:100F9000E5520701C5AD80D000C7E6FF01C7E6FFF7
:100FA00051EC32F0E552E552020EF3CFDBFF030EB7
:100FB000F4CFDBFFDE6ADD6ADECF14F0DDCF15F0A3
:100FC000020EDBCF16F0030EDBCF17F01650145CC9
:100FD000175015582CE2020EDBCF16F0030EDBCFB4
:100FE00017F0DE50165CE96EDD501758EA6EE90620
:100FF000000EEA5A280EE926090EEA22EF50E66EA4
:10100000FC0EDB50040F146E156ADE50145CE96EA2
:10101000DD501558EA6E280EE926090EEA22E5523F
:10102000E750EF6EDF2A010E01E3DB2AC5D7DE6A47
:10103000DD6ADECF14F0DDCF15F0FC0EDB50050FBE
:10104000186E196A020EDB50185C166E030EDB5028
:101050001958176E1650145C175015581DE20701E9
:10106000C5A90BD0DECFE9FFDDCFEAFF280EE926C8
:10107000090EEA22300EEF6E0AD0DECFE9FFDDCF97
:10108000EAFF280EE926090EEA22200EEF6EDF2A7B
:10109000010E01E3DB2ACDD7FC0EDB50050FEA6A17
:1010A000280FE96E090EEA22EF6A0701C4AF09D0E2
:1010B00000C7E6FF01C7E6FFA3EC00F0E552E552EA
:1010C0000DD000C7E6FF01C7E6FF47DDE552E55258
:1010D000020EF3CFDBFF030EF4CFDBFF0A0EE15C61
:1010E00002E2E16AE552E16EE552E7CFD9FF120074
:1010F000D9CFE6FFE1CFD9FF0E0EE126F90EDBCF07
:10110000DEFFDBCFDDFFF80EDB50000802E3070E49
:1011100008D0F80EDB50160802E2170E02D0F80EC7
:10112000DB28E66ED950080FE96EDACFEAFFE55208
:10113000E750EE6EED6A020EDB6A030EDB6AFB0E11
:10114000DBCF14F0FC0EDBCF15F0FD0EDBCF16F07D
:10115000FE0EDBCF17F00C6A0D6A0E6A0F6A14C020
:1011600007F015C008F016C009F017C00AF05AECD5
:1011700028F0010A33E1F90EDBCFE9FFDB2AFA0E92
:10118000DBCFEAFF01E3DB2A2D0EEF6EFB0EDBCF98
:1011900014F0FC0EDBCF15F0FD0EDBCF16F0FE0ECB
:1011A000DBCF17F00C6A0D6A800E0E6EBF0E0F6E4D
:1011B00014C007F015C008F016C009F017C00AF0F7
:1011C00031EC27F0FB0E07C0DBFFFC0E08C0DBFF95
:1011D000FD0E09C0DBFFFE0E0AC0DBFFFB0EDBCFFE
:1011E00014F0FC0EDBCF15F0FD0EDBCF16F0FE0E7B
:1011F000DBCF17F00C6A0D6A0E6A0F6A14C007F095
:1012000015C008F016C009F017C00AF051EC28F01C
:10121000010A4AE1FB0EDBCF14F0FC0EDBCF15F028
:10122000FD0EDBCF16F0FE0EDBCF17F00C6A0D6A59
:10123000800E0E6E3F0E0F6E14C007F015C008F042
:1012400016C009F017C00AF05AEC28F0010A2CE188
:10125000146A156A200E166E410E176ED950FB0FD8
:10126000E96EFF0EDA20EA6EEECF07F0EECF08F05F
:10127000EECF09F0EFCF0AF014C00CF015C00DF05E
:1012800016C00EF017C00FF031EC27F00AC0EDFFCA
:1012900009C0EDFF08C0EDFF07C0EFFF020EDB063F
:1012A000030E01E2DB06B6D7FB0EDBCF14F0FC0E1B
:1012B000DBCF15F0FD0EDBCF16F0FE0EDBCF17F007
:1012C0000C6A0D6A200E0E6E410E0F6E14C007F0F0
:1012D00015C008F016C009F017C00AF05AEC28F043
:1012E000010A2EE0FB0EDBCF14F0FC0EDBCF15F075
:1012F000FD0EDBCF16F0FE0EDBCF17F00C6A0D6A89
:10130000200E0E6E410E0F6E14C007F015C008F0CF
:1013100016C009F017C00AF0DEEC26F0FB0E07C07D
:10132000DBFFFC0E08C0DBFFFD0E09C0DBFFFE0E7D
:101330000AC0DBFF020EDB2A030E01E3DB2AB4D76F
:10134000020EDBCF14F0030EDBCF15F0D950080FDF
:10135000E96EDACFEAFF1450EE261550ED22010EA9
:10136000F36E040EF3CFDBFF050EDB6A040EDBCF5A
:1013700008F0050EDBCF09F019EC26F00A0E07C0C5
:10138000DBFF0B0E08C0DBFF0C0E09C0DBFF0D0EF0
:101390000AC0DBFF040EDBCF14F0050EDBCF15F027
:1013A000080EDBCF16F0090EDBCF17F0155017181B
:1013B000E8AE02D0173404D01650145C17501558FC
:1013C0002EE20A0EDBCF14F00B0EDBCF15F00C0E65
:1013D000DBCF16F00D0EDBCF17F00C6A0D6A200E76
:1013E0000E6E410E0F6E14C007F015C008F016C047
:1013F00009F017C00AF0DEEC26F00A0E07C0DBFF8A
:101400000B0E08C0DBFF0C0E09C0DBFF0D0E0AC07F
:10141000DBFF040EDB2A050E01E3DB2ABBD70A0E35
:10142000DBCF18F00B0EDBCF19F00C0EDBCF1AF070
:101430000D0EDBCF1BF00C6A0D6A0E6A400E0F6EAC
:1014400018C007F019C008F01AC009F01BC00AF054
:10145000DEEC26F007C014F008C015F009C016F045
:101460000AC017F0D950FB0FE96EFF0EDA20EA6EC2
:10147000EECF07F0EECF08F0EECF09F0EFCF0AF095
:1014800014C00CF015C00DF016C00EF017C00FF010
:1014900048EC26F00AC0EDFF09C0EDFF08C0EDFFE3
:1014A00007C0EFFFFB0EDBCF14F0FC0EDBCF15F017
:1014B000FD0EDBCF16F0FE0EDBCF17F00C6A0D6AC7
:1014C000200E0E6E410E0F6E14C007F015C008F00E
:1014D00016C009F017C00AF05AEC28F0010A13E010
:1014E000FB0EDB6AFC0EDB6A800EF36EFD0EF3CFA3
:1014F000DBFF3F0EF36EFE0EF3CFDBFF020EDB2AA7
:10150000030E01E3DB2A020EDBCF14F0030EDBCF68
:1015100015F00001800E15145FE0F90EDBCFE9FF36
:10152000DB2AFA0EDBCFEAFF01E3DB2A300EEF6E97
:10153000F90EDBCFE9FFDB2AFA0EDBCFEAFF01E38E
:10154000DB2A2E0EEF6E080EDBCF14F0090EDBCF78
:1015500015F0800E151414E0020EDBCF16F0030E0A
:10156000DBCF17F0080EDB50165C146E090EDB5053
:101570001758156E020E14C0DBFF030E15C0DBFFFB
:10158000040EDB68050EDB68040EDBCF14F0050EDD
:10159000DBCF15F0020EDBCF16F0030EDBCF17F01A
:1015A00017501518E8AE02D0153404D01450165C4C
:1015B0001550175811E2F90EDBCFE9FFDB2AFA0EBE
:1015C000DBCFEAFF01E3DB2A300EEF6E040EDB0611
:1015D000050E01E2DB06D8D7040EDB6A050EDB6AD6
:1015E000040EDBCF14F0050EDBCF15F0080EDBCFB9
:1015F00016F0090EDBCF17F015501718E8AE02D021
:10160000173404D01650145C1750155801E3ACD0B1
:10161000FB0EDBCF07F0FC0EDBCF08F0FD0EDBCFBF
:1016200009F0FE0EDBCF0AF0EBEC27F0060E08C047
:10163000DBFF070E09C0DBFF300EE76E060EDBCFC7
:1016400014F0070EDBCF15F0E7501426000E15221C
:10165000F90EDBCFE9FFDB2AFA0EDBCFEAFF01E36D
:10166000DB2A14C0EFFF040EDBCF14F0050EDBCF36
:1016700015F0020EDB50141803E1030EDB501518B1
:101680000BE1F90EDBCFE9FFDB2AFA0EDBCFEAFF35
:1016900001E3DB2A2E0EEF6E060EDBCF08F0070EFD
:1016A000DBCF09F019EC26F00A0E07C0DBFF0B0EAA
:1016B00008C0DBFF0C0E09C0DBFF0D0E0AC0DBFF0C
:1016C00007C014F008C015F009C016F00AC017F0E2
:1016D000D950FB0FE96EFF0EDA20EA6EEECF07F06D
:1016E000EECF08F0EECF09F0EFCF0AF014C00CF007
:1016F00015C00DF016C00EF017C00FF047EC26F025
:101700000AC0EDFF09C0EDFF08C0EDFF07C0EFFF05
:10171000146A156A200E166E410E176ED950FB0F13
:10172000E96EFF0EDA20EA6EEECF07F0EECF08F09A
:10173000EECF09F0EFCF0AF014C00CF015C00DF099
:1017400016C00EF017C00FF031EC27F00AC0EDFF05
:1017500009C0EDFF08C0EDFF07C0EFFF040EDB2A54
:10176000050E01E3DB2A3CD7F90EDBCFE9FFFA0EC9
:10177000DBCFEAFFEF6A0E0EE15C02E2E16AE552BE
:10178000E16EE552E7CFD9FF1200D9CFE6FFE1CFF6
:10179000D9FF060EE1260701C49DFB0EDBCF07F043
:1017A000FC0EDBCF08F0FD0EDBCF09F0FE0EDBCF29
:1017B0000AF01AEC28F006C0DEFF07C0DEFF08C002
:1017C000DEFF09C0DDFFDD52DD52F90EDBCF08F090
:1017D000FA0EDBCF09F019EC26F007C014F008C0B0
:1017E00015F009C016F00AC017F0FB0EDBCF1CF095
:1017F000FC0EDBCF1DF0FD0EDBCF1EF0FE0EDBCFAF
:101800001FF0D9CFE9FFDACFEAFFEECF24F0EECF19
:1018100025F0EECF26F0EFCF27F024C006F025C04C
:1018200007F026C008F027C009F02EEC26F007C00C
:1018300020F008C021F009C022F00AC023F020C027
:101840000CF021C00DF022C00EF023C00FF01CC020
:1018500007F01DC008F01EC009F01FC00AF047ECD9
:1018600026F007C018F008C019F009C01AF00AC025
:101870001BF018C00CF019C00DF01AC00EF01BC000
:101880000FF014C007F015C008F016C009F017C01B
:101890000AF031EC27F0EBEC27F0040E08C0DBFF78
:1018A000050E09C0DBFFD60EE66E080EE66ED9CF38
:1018B000E9FFDACFEAFFEECFE6FFEECFE6FFEECFAD
:1018C000E6FFEFCFE6FF07EC2EF0146E060EE15EAA
:1018D00014500701C4AF09D0D60EE66E080EE66EAE
:1018E000A3EC00F0E552E5520CD0D60EE66E080EE1
:1018F000E66EADEC05F0E552E552F3CF16F7F4CF06
:1019000017F70701C4AF06D02E0EE66E61EC00F0AB
:10191000E55205D02E0EE66EE4EC05F0E552E66ADF
:10192000040EDBCFE6FF050EDBCFE6FF7EEC07F013
:10193000E552E552E552060EE15C02E2E16AE5524B
:10194000E16EE552E7CFD9FF1200D9CFE6FFE1CF34
:10195000D9FFE652800EDF6EDF50000813E2FE0E64
:10196000DB50DF1406E0310EE66EE4EC05F0E552E4
:1019700005D0300EE66EE4EC05F0E552DF407F0B5B
:10198000DF6EEAD7E552E552E7CFD9FF1200D9CF93
:10199000E6FFE1CFD9FF020EE126010EDB6AFE0E63
:1019A000DB50F00BE8380F0B300FDF6EDF503908DB
:1019B00003E2070EDF24DF6EFE0EDB500F0B300F4D
:1019C000E76E010EE7CFDBFFDB5039080AE2070EB6
:1019D000146E010EDBCFE7FF1450E726010EE7CFB0
:1019E000DBFF0701C4BF11D0DFCFE6FFE4EC05F059
:1019F000E552010EDBCFE6FFE4EC05F0E552680EA0
:101A0000E66EE4EC05F0E55210D0DFCFE6FF61ECC6
:101A100000F0E552010EDBCFE6FF61EC00F0E5528D
:101A2000680EE66E61EC00F0E552020EE15C02E247
:101A3000E16AE552E16EE552E7CFD9FF1200D9CF56
:101A4000E6FFE1CFD9FFFB0EDBCF07F0FC0EDBCFCB
:101A500008F0FD0EDBCF09F0FE0EDBCF0AF00A34F2
:101A6000000E0A1809E6D880000E0754000E08542C
:101A7000000E0954000E0A540CE2D950FB0FE96E17
:101A8000FF0EDA20EA6EEE06000EEE5AEE5AEE5A1D
:101A9000DAD7E552E7CFD9FF1200D9CFE6FFE1CF81
:101AA000D9FF020EE126DE6ADD6ADECF14F0DDCF5B
:101AB00015F0FE0EDB50000115AE02D0D89003D019
:101AC000145C000E15580AE2200EE66EE4EC05F0F8
:101AD000E552DF2A010E01E3DB2AE7D7020EE15CC3
:101AE00002E2E16AE552E16EE552E7CFD9FF12006A
:101AF0000F01426B428F428B42890901D60E266F3D
:101B0000080E276F370E146E660E156E166A14C017
:101B1000E6FF15C0E6FF16C0E6FF26C9E6FF27C9A7
:101B2000E6FF38EC32F0176E050EE15E1750070144
:101B3000C4AF0ED0020EE66EE1EC00F0E55226C90D
:101B4000E6FF27C9E6FFA3EC00F0E552E5520ED010
:101B500026C9E6FF27C9E6FFADEC05F0E552E552E0
:101B6000F3CF16F7F4CF17F7F4EC05F0E80EE66EB6
:101B7000030EE66EE66AE66A62DFE552E552E5527A
:101B8000E5520F01418F419D418B41874195419124
:101B9000406B12000F013D93799E7998C90E796EC2
:101BA0003D95789E7898DD0E786E778A778877965F
:101BB000779477927790A09CA09AA28CA28A120028
:101BC000806A0F01386B38813883388538870F0E6B
:101BD000926E8168396B030E936E020E616EF19EF8
:101BE00082683A6B800E946E949C948E836A3B6BF1
:101BF000BF0E956E846A3C6B966A606A1200C28062
:101C0000C19EC08EC08AC088C096C082C094C09059
:101C1000C196C194C192C1901200D9CFE6FFE1CF25
:101C2000D9FF020EE126FD0EDBCF14F0FE0EDBCF56
:101C300015F0D89014361536D89014361536010E96
:101C40001424C26E0A0EE66E20EC33F0E55239EC35
:101C500033F034EC33F0000901E0FBD72BEC33F028
:101C6000F3CFDEFFF4CFDDFFDECF14F0DDCF15F0D4
:101C700014C0F3FF15C0F4FF020EE15C03E200D0D4
:101C8000E16AE552E16EE552E7CFD9FF1200CD9E41
:101C9000CD9CCD8ACD88CD96CD94CD82CD90CC9E55
:101CA000CC9ACC92CC909F80D08E9D90DB0EE66E2D
:101CB0000B0EE66E7EEC32F0E552E5529E90F28C11
:101CC000CD90F28EF28C0701CA6BCB6B1200D9CF8C
:101CD000E6FFE1CFD9FF020EE126DE6ADD6AFB0EE8
:101CE000DBCFF6FFDB2AFC0EDBCFF7FF01E3DB2ABD
:101CF0000800F550E66EFD0EDBCFE9FFDB2AFE0E95
:101D0000DBCFEAFF01E3DB2AE552E750EF6EDF2A83
:101D1000010E01E3DB2ADECF14F0DDCF15F0D89001
:101D2000155004E6000E145C010E1558D8E3020E9F
:101D3000E15C02E2E16AE552E16EE552E7CFD9FFEC
:101D40001200D9CFE6FFE1CFD9FF020EE126DE6A0D
:101D5000DD6AFB0EDBCFF6FFDB2AFC0EDBCFF7FFE5
:101D600001E3DB2A0800F550E66EFF0EE76EFD0E7C
:101D7000DBCF14F0FE0EDBCF15F0E7501426000E7B
:101D80001522DE50145CE96EDD501558EA6EE552FE
:101D9000E750EF6EDF2A010E01E3DB2ADECF14F0FD
:101DA000DDCF15F0D890155004E6000E145C010E3E
:101DB0001558CFE3020EE15C02E2E16AE552E16E02
:101DC000E552E7CFD9FF1200D9CFE6FFE1CFD9FF27
:101DD000FB0EDBCF14F0FC0EDBCF15F0FD0EDBCFDE
:101DE00016F0FE0EDBCF17F014C006F015C007F09A
:101DF00016C008F017C009F02EEC26F007C064F7F3
:101E000008C065F709C066F70AC067F7FC0EF66EF2
:101E1000560EF76E0900F5CF68F70900F5CF69F7A0
:101E20000900F5CF6AF70800F5CF6BF768C70CF02B
:101E300069C70DF06AC70EF06BC70FF064C707F0F3
:101E400065C708F066C709F067C70AF0DEEC26F040
:101E500007C060F708C061F709C062F70AC063F7FE
:101E600060C7E6FF61C7E6FF62C7E6FF63C7E6FF3C
:101E700028EC31F0E552E552E552E55206C014F087
:101E800007C015F008C016F009C017F014C007F01D
:101E900015C008F016C009F017C00AF01AEC28F0B7
:101EA00006C0BCF707C0BDF708C0BEF709C0BFF742
:101EB0000701C48F020EE66EE1EC00F0E552070167
:101EC000090E901901E1915140E11CC714F01DC7A2
:101ED00015F00A0E0D6E0E6A14C008F015C009F058
:101EE0009EEC27F008C014F009C015F0300E142441
:101EF000E66E61EC00F0E5521CC714F01DC715F04A
:101F00000A0E0D6E0E6A14C008F015C009F09EECA2
:101F100027F004C014F005C015F0300E1424E66E4E
:101F200061EC00F0E552200EE66E61EC00F0E55247
:101F3000200EE66E61EC00F0E552060EE66E020E33
:101F4000E66EC4EC00F0E552E552010EE66E26C9DD
:101F5000E6FF27C9E6FF64C7E6FF65C7E6FF66C779
:101F6000E6FF67C7E6FF78EC08F0146E070EE15E47
:101F7000145026C9E6FF27C9E6FFA3EC00F0E5529E
:101F8000E552200EE66E61EC00F0E552480EE66E7A
:101F900061EC00F0E5527A0EE66E61EC00F0E5527D
:101FA0000701C49F26C9E6FF27C9E6FFADEC05F08F
:101FB000E552E552F3CF16F7F4CF17F7480EE66E69
:101FC000E4EC05F0E5527A0EE66EE4EC05F0E5523D
:101FD000F4EC05F00701C48FBCC7D7F7BDC7D6F72F
:101FE000BEC7D5F7B86BB96BBA6BBB6BE552E7CF21
:101FF000D9FF12000701600E046F000E056F04C7C1
:1020000002F705C703F7CE6BCF6B116B076B12009E
:102010000701C4AF05D0010EE66EE1EC00F0E55219
:10202000010EE66EE66AE3EC06F0E552E5520701C2
:10203000126B136B000E125D010E135946E2FC0E7B
:102040001225F66E520E1321F76E0800F5CF18F028
:1020500018C009F006EC26F007C014F008C015F00F
:1020600009C016F00AC017F00C6A0D6A0E6A410E1C
:102070000F6E14C007F015C008F016C009F017C0A5
:102080000AF0DEEC26F007C070F708C071F709C04F
:1020900072F70AC073F770C707F071C708F072C70C
:1020A00009F073C70AF0C4EC27F00950E66E000E81
:1020B00007011225E96E060E1321EA6EE552E7507C
:1020C000EF6E122B000E1323B5D712000701C4AF19
:1020D00005D0010EE66EE1EC00F0E552020EE66E70
:1020E000E66AE3EC06F0E552E5520701126B136B6A
:1020F000800E125D000E13590CE2000E1225E96EDF
:10210000060E1321EA6E1F0EEF6E122B000E132324
:10211000EFD7800E126F136B000E125D010E135974
:102120000BE2000E1225E96E060E1321EA6EEF6A2D
:10213000122B000E1323F0D712000701C4AF05D0F5
:10214000010EE66EE1EC00F0E552030EE66EE66A83
:10215000E3EC06F0E552E5520701126B136B800EBB
:10216000125D000E135940E212C708F013C709F0C0
:1021700017EC26F007C014F008C015F009C016F0DF
:102180000AC017F00C6A0D6A800E0E6E400E0F6EBC
:1021900014C007F015C008F016C009F017C00AF007
:1021A000DEEC26F007C070F708C071F709C072F7BF
:1021B0000AC073F770C707F071C708F072C709F05B
:1021C00073C70AF0C4EC27F00950E66E000E070151
:1021D0001225E96E060E1321EA6EE552E750EF6E06
:1021E000122B000E1323BBD7800E126F136B000E41
:1021F000125D010E135949E212C718F013C719F006
:10220000FF0ED8801856000E195618C008F019C0D5
:1022100009F017EC26F007C014F008C015F009C04B
:1022200016F00AC017F00C6A0D6A800E0E6E400E92
:102230000F6E14C007F015C008F016C009F017C0E3
:102240000AF0DEEC26F007C070F708C071F709C08D
:1022500072F70AC073F770C707F071C708F072C74A
:1022600009F073C70AF0C4EC27F00950E66E000EBF
:1022700007011225E96E060E1321EA6EE552E750BA
:10228000EF6E122B000E1323B2D712000701C4AF5A
:1022900005D0010EE66EE1EC00F0E552040EE66EAC
:1022A000E66AE3EC06F0E552E5520701126B136BA8
:1022B000000E125D010E13593FE212C708F013C75A
:1022C00009F017EC26F007C014F008C015F009C09B
:1022D00016F00AC017F00C6A0D6A0E6A410E0F6EF6
:1022E00014C007F015C008F016C009F017C00AF0B6
:1022F000DEEC26F007C070F708C071F709C072F76E
:102300000AC073F770C707F071C708F072C709F009
:1023100073C70AF0C4EC27F00950E66E000E0701FF
:102320001225E96E060E1321EA6EE552E750EF6EB4
:10233000122B000E1323BCD712000701C4AF05D027
:10234000010EE66EE1EC00F0E552050EE66EE66A7F
:10235000E3EC06F0E552E5520701126B136B000E39
:10236000125D010E135948E212C718F013C719F095
:10237000FF0ED8801856000E195618C008F019C064
:1023800009F017EC26F007C014F008C015F009C0DA
:1023900016F00AC017F00C6A0D6A0E6A410E0F6E35
:1023A00014C007F015C008F016C009F017C00AF0F5
:1023B000DEEC26F007C070F708C071F709C072F7AD
:1023C0000AC073F770C707F071C708F072C709F049
:1023D00073C70AF0C4EC27F00950E66E000E07013F
:1023E0001225E96E060E1321EA6EE552E750EF6EF4
:1023F000122B000E1323B3D71200D9CFE6FFE1CF83
:10240000D9FF020EE1261EC714F01FC715F0D890A1
:1024100015321432D8901532143214C0DEFF15C0B4
:10242000DDFF0701C4AF05D0010EE66EE1EC00F060
:10243000E552060EE66EE66AE3EC06F0E552E5527A
:10244000D9CFE9FFDACFEAFF000ED880EE54000EB4
:10245000ED5435E2DECF14F0DDCF15F0FF0E145C45
:10246000000E15582CE20701126B136BDECF14F02F
:10247000DDCF15F01450125D155013590CE2000E0B
:102480001225E96E060E1321EA6E1F0EEF6E122B57
:10249000000E1323EBD7DECF12F7DDCF13F7000EBC
:1024A000125D010E13590BE2000E1225E96E060EA5
:1024B0001321EA6EEF6A122B000E1323F0D7020EDF
:1024C000E15C02E2E16AE552E16EE552E7CFD9FF55
:1024D0001200200EE66E61EC00F0E552060EE66E8C
:1024E000020EE66EC4EC00F0E552E5529CC706F021
:1024F0009DC707F09EC708F09FC709F02EEC26F095
:1025000007C070F708C071F709C072F70AC073F707
:102510000901D60E266F080E276F010EE66E26C93A
:10252000E6FF27C9E6FF70C7E6FF71C7E6FF72C77F
:10253000E6FF73C7E6FF78EC08F0146E070EE15E65
:10254000145007010B0E901901E191511BE1030E8C
:10255000E66E020EE66EC4EC00F0E552E55226C9C6
:10256000E6FF27C9E6FF51EC32F0E552E552F3CF22
:1025700014F7F4CF15F707010A0ED8801457000E90
:1025800015571AD026C9E6FF27C9E6FF51EC32F0ED
:10259000E552E552F3CF14F7F4CF15F70701070E14
:1025A000D8801457000E1557060EE66E020EE66E22
:1025B000C4EC00F0E552E552070114C714F015C74A
:1025C00015F01407000E155BD8801454000E155436
:1025D00006E2200EE66E61EC00F0E552EDD726C96A
:1025E000E6FF27C9E6FFA3EC00F0E552E552200E16
:1025F000E66E61EC00F0E552480EE66E61EC00F02C
:10260000E5527A0EE66E61EC00F0E552880EE66E59
:10261000130EE66EE66AE66A1FEC0DF0E552E5522F
:10262000E552E5521200D9CFE6FFE1CFD9FF080EFF
:10263000E126FB0EDBCF9CF7FC0EDBCF9DF7FD0EFA
:10264000DBCF9EF7FE0EDBCF9FF781A0FED7060EF5
:10265000DB6A070EDB6ACD909E900701C66BC76BE5
:10266000000EE66EE66A0DEC0EF0E552E552F3CF91
:10267000DEFFF4CFDDFFD00EE66E070EE66EE66AF3
:10268000E66A1FEC0DF0E552E552E552E552D9CF6E
:10269000E9FFDACFEAFFBC0ED880EE54020EED540B
:1026A0001CE3DECF14F0DDCF15F02C0E145C010E10
:1026B000155813E38D848D808D92E66A020EE66EC6
:1026C000C4EC00F0E552E5523D0EE66E61EC00F020
:1026D000E552FFDE0701C66BC76BD9CFE9FFDACF42
:1026E000EAFFBC0ED880EE54020EED5401E3DDD0BB
:1026F0008D948D828D800701C66BC76BD9CFE9FFA2
:10270000DACFEAFFBC0ED880EE54020EED5401E39E
:10271000CCD0000EE66EE66A0DEC0EF0E552E55206
:10272000F3CFDEFFF4CFDDFF0701C62B000EC7237A
:10273000C6C714F0C7C715F0030ED890153214326F
:10274000E804FBE1060E14C0DBFF070E15C0DBFF3B
:10275000D950060FE96EDACFEAFF0A0ED880EE54A0
:10276000000EED5407E20A0EF36E060EF3CFDBFF08
:10277000070EDB6A07010B0E901901E191511DE173
:10278000060EDBCFE9FF070EDBCFEAFF020ED89083
:10279000E936EA36E806FBE1A80EE926080EEA2249
:1027A000020EEECFDBFF030EEECFDBFF040EEECF0B
:1027B000DBFF050EEECFDBFF1ED0060EDBCFE9FF01
:1027C000070EDBCFEAFF010ED890E936EA36E806BD
:1027D000FBE1920EE926080EEA22EECF14F0EFCFCD
:1027E00015F0020E14C0DBFF030E15C0DBFF040E54
:1027F000DB6A050EDB6AD950020FE96EDACFEAFF19
:1028000007019C51EE24146E9D51EE20156E9E51D1
:10281000EE20166E9F51EE20176EF30EDBCF07F001
:10282000F40EDBCF08F0F50EDBCF09F0F60EDBCFB0
:102830000AF017500A18E8AE02D00A3408D0075040
:10284000145C08501558095016580A50175812E2CF
:10285000D950020FE96EDACFEAFF9C51EE249C6F4B
:102860009D51EE209D6F9E51EE209E6F9F51EE2058
:102870009F6F0CD0F30EDBCF9CF7F40EDBCF9DF7F0
:10288000F50EDBCF9EF7F60EDBCF9FF7C48FE66A1F
:10289000020EE66EC4EC00F0E552E5523E0EE66E26
:1028A00061EC00F0E55215DE29D7DECF14F0DDCF64
:1028B00015F02C0E145C010E155801E3D6D08D8452
:1028C0008D828D900701C66BC76BDECF14F0DDCF14
:1028D00015F02C0E145C010E155801E3C6D007014B
:1028E000C62B000EC723E66EE66A0DEC0EF0E5522D
:1028F000E552F3CFDEFFF4CFDDFFC6C714F0C7C744
:1029000015F0030ED89015321432E804FBE1060EE0
:1029100014C0DBFF070E15C0DBFFD950060FE96EB0
:10292000DACFEAFF0A0ED880EE54000EED5407E22B
:102930000A0EF36E060EF3CFDBFF070EDB6A07010C
:102940000B0E901901E191511DE1060EDBCFE9FF5D
:10295000070EDBCFEAFF020ED890E936EA36E8062A
:10296000FBE1A80EE926080EEA22020EEECFDBFFFD
:10297000030EEECFDBFF040EEECFDBFF050EEECF36
:10298000DBFF1ED0060EDBCFE9FF070EDBCFEAFF31
:10299000010ED890E936EA36E806FBE1920EE92608
:1029A000080EEA22EECF14F0EFCF15F0020E14C09D
:1029B000DBFF030E15C0DBFF040EDB6A050EDB6ACE
:1029C000F70EDBCF14F0F80EDBCF15F0F90EDBCFEE
:1029D00016F0FA0EDBCF17F0D950020FE96EDACFFE
:1029E000EAFFEE501426EE501522EE501622EE505D
:1029F0001722175007019F19E8AE02D09F3508D063
:102A00009C51145C9D5115589E5116589F51175852
:102A100012E2D950020FE96EDACFEAFFEE509C5D68
:102A20009C6FEE509D599D6FEE509E599E6FEE50DB
:102A30009F599F6F0CD0F70EDBCF9CF7F80EDBCFC2
:102A40009DF7F90EDBCF9EF7FA0EDBCF9FF7E66A14
:102A5000020EE66EC4EC00F0E552E5523C0EE66E66
:102A600061EC00F0E55235DD30D781B0F0D5880E4D
:102A7000E66E130EE66EE66AE66A1FEC0DF0E552AE
:102A8000E552E552E55281A0FED70701C49F090136
:102A9000D60E266F080E276F9CC706F09DC707F05D
:102AA0009EC708F09FC709F02EEC26F007C070F70C
:102AB00008C071F709C072F70AC073F7010EE66E1D
:102AC00026C9E6FF27C9E6FF70C7E6FF71C7E6FF24
:102AD00072C7E6FF73C7E6FF78EC08F0146E070EC6
:102AE000E15E145026C9E6FF27C9E6FFADEC05F00C
:102AF000E552E552F3CF14F0F4CF15F0166A176AD9
:102B000015AE02D016681768020E14C0DBFF030E64
:102B100015C0DBFF040E16C0DBFF050E17C0DBFF80
:102B2000F4EC05F00701C48F9CC706F09DC707F0C1
:102B30009EC708F09FC709F0080EE15C03E200D0D1
:102B4000E16AE552E16EE552E7CFD9FF1200200EAF
:102B5000E66E61EC00F0E552070EE66E020EE66EE0
:102B6000C4EC00F0E552E5529AC708F09BC709F0A3
:102B700017EC26F007C018F008C019F009C01AF0C9
:102B80000AC01BF00C6A0D6AC80E0E6E420E0F6E64
:102B900018C007F019C008F01AC009F01BC00AF0ED
:102BA00031EC27F007C014F008C015F009C016F08A
:102BB0000AC017F00C6A0D6A800E0E6E440E0F6E7E
:102BC00014C007F015C008F016C009F017C00AF0CD
:102BD000DEEC26F007C06CF708C06DF709C06EF791
:102BE0000AC06FF7010EE66E26C9E6FF27C9E6FFA9
:102BF0006CC7E6FF6DC7E6FF6EC7E6FF6FC7E6FF6F
:102C000078EC08F0146E070EE15E145026C9E6FF5A
:102C100027C9E6FFA3EC00F0E552E552100EE66E80
:102C2000270EE66EE66AE66A1FEC0DF0E552E55205
:102C3000E552E5521200D9CFE6FFE1CFD9FF040EED
:102C4000E126FD0EDBCF9AF7FE0EDBCF9BF7CD9092
:102C50000701C48F020EE66EE1EC00F0E5520701B9
:102C6000C66BC76B146B156B000EE66EE66A0DEC57
:102C70000EF0E552E552F3CFDEFFF4CFDDFFD00ECC
:102C8000E66E070EE66EE66AE66A1FEC0DF0E552A8
:102C9000E552E552E552D9CFE9FFDACFEAFFEE0E71
:102CA000D880EE54020EED541EE3DECF14F0DDCFDB
:102CB00015F0FA0E145C000E155815E38D848D8006
:102CC0008D92E66A020EE66EC4EC00F0E552E55223
:102CD0003D0EE66E61EC00F0E55239DF0701C66B90
:102CE000C76B146B156BD9CFE9FFDACFEAFFEE0E95
:102CF000D880EE54020EED5401E399D00701C66B63
:102D0000C76B8D948D828D80D9CFE9FFDACFEAFF32
:102D1000EE0ED880EE54020EED5401E388D0000E82
:102D2000E66EE66A0DEC0EF0E552E552F3CFDEFFFB
:102D3000F4CFDDFF0701C62B000EC723C6C714F072
:102D4000C7C715F0030ED89015321432E804FBE122
:102D500014C014F715C015F707010A0ED8801455D2
:102D6000000E155503E20A0E146F156B0B0E901929
:102D700001E1915115E114C7E9FF15C7EAFF010E02
:102D8000D890E936EA36E806FBE17C0EE926080E23
:102D9000EA22020EEECFDBFF030EEDCFDBFF14D0F5
:102DA00014C7E9FF15C7EAFF010ED890E936EA36E5
:102DB000E806FBE17C0EE926080EEA22020EEECFC1
:102DC000DBFF030EEDCFDBFF020EDB5007019A2580
:102DD0000001146E030EDB5007019B210001156EEC
:102DE000F90EDBCF16F0FA0EDBCF17F01650145C9D
:102DF0001750155808E2020EDB5007019A27030E00
:102E0000DB509B2306D0F90EDBCF9AF7FA0EDBCF0F
:102E10009BF7E66A020EE66EC4EC00F0E552E5525E
:102E20003E0EE66E61EC00F0E55291DE6DD7DECF2E
:102E300014F0DDCF15F0FA0E145C000E155801E306
:102E400099D00701C66BC76BDECF14F0DDCF15F04C
:102E5000FA0E145C000E155801E38CD08D848D821F
:102E60008D900701C62B000EC723E66EE66A0DECB7
:102E70000EF0E552E552F3CFDEFFF4CFDDFFC6C71B
:102E800014F0C7C715F0030ED89015321432E804B9
:102E9000FBE114C014F715C015F707010A0ED8801E
:102EA0001455000E155503E20A0E146F156B0B0E28
:102EB000901901E1915115E114C7E9FF15C7EAFF27
:102EC000010ED890E936EA36E806FBE17C0EE926E9
:102ED000080EEA22020EEECFDBFF030EEDCFDBFF82
:102EE00014D014C7E9FF15C7EAFF010ED890E936E0
:102EF000EA36E806FBE17C0EE926080EEA22020E1D
:102F0000EECFDBFF030EEDCFDBFF020EDB50070140
:102F10009A5D0001146E030EDB5007019B590001FE
:102F2000156EFB0EDBCF16F0FC0EDBCF17F0145046
:102F3000165C1550175808E2020EDB5007019A5F25
:102F4000030EDB509B5B06D0FB0EDBCF9AF7FC0E2B
:102F5000DBCF9BF70701C48FE66A020EE66EC4EC76
:102F600000F0E552E5523E0EE66E61EC00F0E552EF
:102F7000EEDD6AD781B073D6880EE66E130EE66E6C
:102F8000E66AE66A1FEC0DF0E552E552E552E552BD
:102F900081A0FED70701C49F9AC708F09BC709F01C
:102FA00017EC26F007C018F008C019F009C01AF095
:102FB0000AC01BF00C6A0D6AC80E0E6E420E0F6E30
:102FC00018C007F019C008F01AC009F01BC00AF0B9
:102FD00031EC27F007C014F008C015F009C016F056
:102FE0000AC017F00C6A0D6A800E0E6E440E0F6E4A
:102FF00014C007F015C008F016C009F017C00AF099
:10300000DEEC26F007C06CF708C06DF709C06EF75C
:103010000AC06FF7020EE66E26C9E6FF27C9E6FF73
:103020006CC7E6FF6DC7E6FF6EC7E6FF6FC7E6FF3A
:1030300078EC08F0146E070EE15E145026C9E6FF26
:1030400027C9E6FFADEC05F0E552E552020EF3CFDD
:10305000DBFF030EF4CFDBFFF4EC05F00701C48FB8
:103060009AC7F3FF9BC7F4FF040EE15C03E200D0B4
:10307000E16AE552E16EE552E7CFD9FF1200D9CF00
:10308000E6FFE1CFD9FF020EE1260701C48FE66E0D
:10309000E1EC00F0E5520701CA6BCB6B47EC0EF098
:1030A000CD809E909D80DE6ADD6AE66A020EE66E45
:1030B000C4EC00F0E552E552CAC714F0CBC715F0D6
:1030C000330ED8801456000E15561450E66E61EC7F
:1030D00000F0E55281B015D09D90010EDE6EDD6AE4
:1030E000030E0701CA6FCB6B010EE66E020EE66E91
:1030F000C4EC00F0E552E552200EE66E61EC00F003
:10310000E5520701030ECA5D000ECB59CEE39D9038
:10311000CD909E90C66BC76B81A0FED7DECF14F01A
:10312000DDCF15F014C0F3FF15C0F4FF020EE15C13
:1031300003E200D0E16AE552E16EE552E7CFD9FF44
:103140001200D9CFE6FFE1CFD9FF040EE126A09C03
:10315000A09A0701C48F010E921901E1935128E151
:10316000902B000E9123913504E290510B08000E34
:10317000915503E2010E906F916B980EE66E3A0E38
:10318000E66EE66AE66A1FEC0DF0E552E552E5529E
:10319000E552440EE66EE4EC05F0E5520A0EE66EEA
:1031A000E4EC05F0E5520D0EE66EE4EC05F0E552B8
:1031B0000701010E941901E1955124E19007000ED9
:1031C000915B9051911103E10B0E906F916B980EF2
:1031D000E66E3A0EE66EE66AE66A1FEC0DF0E55220
:1031E000E552E552E552470EE66EE4EC05F0E55295
:1031F0000A0EE66EE4EC05F0E5520D0EE66EE4EC28
:1032000005F0E5520B0E0701901901E1915102E121
:103210005FEF1DF00A0E901901E1915101E177D3A2
:10322000090E901901E1915101E1D0D1080E9019D8
:1032300001E1915101E1C7D1070E901901E19151CE
:1032400001E1BED1060E901901E191512FE0050E6A
:10325000901901E1915126E0040E901901E191517C
:103260001DE0030E901901E1915114E0020E901936
:1032700001E191510BE0010E901901E1915102E041
:1032800093EF1EF008EC10F093EF1EF066EC10F0D8
:1032900093EF1EF09DEC10F093EF1EF046EC11F052
:1032A00093EF1EF09DEC11F093EF1EF0FDEC11F08A
:1032B0000701C48F020EE66EE1EC00F0E552010E4C
:1032C000E66E26C9E6FF27C9E6FF64C7E6FF65C7C5
:1032D000E6FF66C7E6FF67C7E6FF78EC08F0146E06
:1032E000070EE15E145026C9E6FF27C9E6FFA3ECEE
:1032F00000F0E552E552200EE66E61EC00F0E5527A
:10330000480EE66E61EC00F0E5527A0EE66E61EC76
:1033100000F0E5520701C49F26C9E6FF27C9E6FF72
:10332000ADEC05F0E552E552F3CF16F7F4CF17F701
:10333000480EE66EE4EC05F0E5527A0EE66EE4EC3B
:1033400005F0E5529CDE020EF3CFDBFF030EF4CF57
:10335000DBFF020EDBCF14F0030EDBCF15F01534CC
:1033600004E214500008000E155401E398D0070140
:10337000C48F010EE66EE1EC00F0E552070EE66E3A
:10338000E66AE3EC06F0E552E552020EE66EE1EC89
:1033900000F0E552070EE66E020EE66EC4EC00F099
:1033A000E552E5521EC708F01FC709F017EC26F0DA
:1033B00007C018F008C019F009C01AF00AC01BF0C5
:1033C0000C6A0D6AC80E0E6E420E0F6E18C007F022
:1033D00019C008F01AC009F01BC00AF031EC27F040
:1033E00007C014F008C015F009C016F00AC017F0A5
:1033F0000C6A0D6A800E0E6E440E0F6E14C007F03C
:1034000015C008F016C009F017C00AF0DEEC26F06F
:1034100007C06CF708C06DF709C06EF70AC06FF7F8
:10342000020EE66E26C9E6FF27C9E6FF6CC7E6FF77
:103430006DC7E6FF6EC7E6FF6FC7E6FF78EC08F0E2
:10344000146E070EE15E145026C9E6FF27C9E6FF99
:10345000A3EC00F0E552E552DE6ADD6A500EE66E3E
:10346000C30EE66EE66AE66A1FEC0DF0E552E55221
:10347000E552E552FE0EE66E030EE66E020EE66EB5
:10348000E66A1EC7E6FF1FC7E6FF1BEC16F0146EC8
:10349000060EE15E1450F3CF1EF7F4CF1FF70701BD
:1034A000C48F010EE66EE1EC00F0E552060EE66E0A
:1034B000E66AE3EC06F0E552E552FDEC11F0020E8F
:1034C000E66EE1EC00F0E552070EE66E020EE66EE7
:1034D000C4EC00F0E552E5521EC708F01FC709F022
:1034E00017EC26F007C018F008C019F009C01AF050
:1034F0000AC01BF00C6A0D6AC80E0E6E420E0F6EEB
:1035000018C007F019C008F01AC009F01BC00AF073
:1035100031EC27F007C014F008C015F009C016F010
:103520000AC017F00C6A0D6A800E0E6E440E0F6E04
:1035300014C007F015C008F016C009F017C00AF053
:10354000DEEC26F007C06CF708C06DF709C06EF717
:103550000AC06FF7020EE66E26C9E6FF27C9E6FF2E
:103560006CC7E6FF6DC7E6FF6EC7E6FF6FC7E6FFF5
:1035700078EC08F0146E070EE15E145026C9E6FFE1
:1035800027C9E6FFA3EC00F0E552E5520701C49F0E
:10359000070EE66EE66AE3EC06F0E552E55226C950
:1035A000E6FF27C9E6FFADEC05F0E552E552F3CFA3
:1035B00016F7F4CF17F7F4EC05F00701C48FB3D377
:1035C000080E906F916B090E906F916B010EE66E75
:1035D000E1EC00F0E552090EE66EE66AE3EC06F077
:1035E000E552E5521CC7E9FF1DC7EAFFD890E9364E
:1035F000EA36FC0EE926070EEA22EECF39F9EFCFC4
:103600003AF909013B6B3C6B020EE66EE1EC00F00F
:10361000E5521CC714F01DC715F00A0E0D6E0E6A98
:1036200014C008F015C009F09EEC27F008C014F093
:1036300009C015F0300E1424E66E61EC00F0E5527E
:103640001CC714F01DC715F00A0E0D6E0E6A14C0CB
:1036500008F015C009F09EEC27F004C014F005C076
:1036600015F0300E1424E66E61EC00F0E552200EE9
:10367000E66E61EC00F0E552200EE66E61EC00F0C3
:10368000E552060EE66E020EE66EC4EC00F0E55260
:10369000E55239C906F03AC907F03BC908F03CC900
:1036A00009F02EEC26F007C064F708C065F709C0E2
:1036B00066F70AC067F7010EE66E26C9E6FF27C95E
:1036C000E6FF64C7E6FF65C7E6FF66C7E6FF67C7B4
:1036D000E6FF78EC08F0146E070EE15E145026C980
:1036E000E6FF27C9E6FFA3EC00F0E552E552200E05
:1036F000E66E61EC00F0E552480EE66E61EC00F01B
:10370000E5527A0EE66E61EC00F0E552B8DC020E8E
:10371000F3CFDBFF030EF4CFDBFF020EDBCF14F0A1
:10372000030EDBCF15F0153404E214500008000E30
:10373000155401E3EBD0DE6ADD6A020EE66EE1ECC1
:1037400000F0E552000EE66EE66A0DEC0EF0E55272
:10375000E552F3CF96F7F4CF97F70701EE0ED88036
:103760009655020E97550DE21C2B000E1D231D359C
:1037700004E21C513F08000E1D5503E2010E1C6FB0
:103780001D6BFA0E965D000E97590FE21C07000E96
:103790001D5B010E1DAF02D0D89003D01C5D000E42
:1037A0001D5903E23F0E1C6F1D6B1CC7E9FF1DC7AF
:1037B000EAFFD890E936EA36FC0EE926070EEA223F
:1037C000EECF39F9EFCF3AF909013B6B3C6B020EB2
:1037D000E66EE1EC00F0E5521CC714F01DC715F0D1
:1037E0000A0E0D6E0E6A14C008F015C009F09EECAA
:1037F00027F008C014F009C015F0300E1424E66E4E
:1038000061EC00F0E5521CC714F01DC715F00A0E5C
:103810000D6E0E6A14C008F015C009F09EEC27F07A
:1038200004C014F005C015F0300E1424E66E61ECEF
:1038300000F0E552200EE66E61EC00F0E552200E3D
:10384000E66E61EC00F0E552060EE66E020EE66EE4
:10385000C4EC00F0E552E55239C906F03AC907F068
:103860003BC908F03CC909F02EEC26F007C064F70C
:1038700008C065F709C066F70AC067F7010EE66E73
:1038800026C9E6FF27C9E6FF64C7E6FF65C7E6FF6E
:1038900066C7E6FF67C7E6FF78EC08F0146E070E10
:1038A000E15E145026C9E6FF27C9E6FFA3EC00F04D
:1038B000E552E552200EE66E61EC00F0E552480E4E
:1038C000E66E61EC00F0E5527A0EE66E61EC00F017
:1038D000E552F00EE66E490EE66E020EE66EE66A00
:1038E0001FEC0DF0E552E552E552E55281B02AD7C2
:1038F000880EE66E130EE66EE66AE66A1FEC0DF0C1
:10390000E552E552E552E55281A0FED70CD2010EF8
:10391000E66EE1EC00F0E5520A0EE66EE66AE3ECD4
:1039200006F0E552E552020EE66EE1EC00F0E552DB
:103930003FEC18F0020EF3CFDBFF030EF4CFDBFFFA
:10394000020EDBCF14F0030EDBCF15F0153404E2CA
:1039500014500008000E15542FE2A80EE66E610EFA
:10396000E66EE66AE66A010EE66EE66AE66AE66A10
:1039700039C9E6FF3AC9E6FF3BC9E6FF3CC9E6FFA5
:1039800013EC13F0146E0C0EE15E145006C039F9FE
:1039900007C03AF908C03BF909C03CF939C9E6FF4C
:1039A0003AC9E6FF3BC9E6FF3CC9E6FFE4EC0EF08E
:1039B000E552E552E552E5520701C48F020EE66E6C
:1039C000E1EC00F0E55239C906F03AC907F03BC90D
:1039D00008F03CC909F02EEC26F007C064F708C0D7
:1039E00065F709C066F70AC067F70901D60E266FAA
:1039F000080E276F010EE66E26C9E6FF27C9E6FF0F
:103A000064C7E6FF65C7E6FF66C7E6FF67C7E6FF70
:103A100078EC08F0146E070EE15E145026C9E6FF3C
:103A200027C9E6FF51EC32F0E552E552F3CF16F725
:103A3000F4CF17F70701070ED8801657000E175757
:103A4000060EE66E020EE66EC4EC00F0E552E5529C
:103A5000070116C714F017C715F01607000E175BFD
:103A6000D8801454000E155406E2200EE66E61EC68
:103A700000F0E552EDD726C9E6FF27C9E6FFA3EC23
:103A800000F0E552E552200EE66E61EC00F0E552E2
:103A9000480EE66E61EC00F0E5527A0EE66E61ECDF
:103AA00000F0E552500EE66EC30EE66EE66AE66A78
:103AB0001FEC0DF0E552E552E552E55234D1010E0E
:103AC000E66EE1EC00F0E5520B0EE66EE66AE3EC22
:103AD00006F0E552E552020EE66EE1EC00F0E5522A
:103AE000E66A020EE66EC4EC00F0E552E55209010A
:103AF000D60E266F080E276F020EE66E26C9E6FF69
:103B000027C9E6FF80C7E6FF81C7E6FF82C7E6FF59
:103B100083C7E6FF78EC08F0146E070EE15E1450E0
:103B200026C9E6FF27C9E6FFA3EC00F0E552E552FF
:103B30003FEC18F0020EF3CFDBFF030EF4CFDBFFF8
:103B4000020EDBCF14F0030EDBCF15F0153404E2C8
:103B500014500008000E155401E3E4D080C7E6FFBE
:103B600081C7E6FF82C7E6FF83C7E6FF28EC31F096
:103B7000E552E552E552E55206C014F007C015F0D3
:103B800008C016F009C017F014C007F015C008F0FF
:103B900016C009F017C00AF01AEC28F006C0A4F706
:103BA00007C0A5F708C0A6F709C0A7F7E66A2D0E5B
:103BB000E66E310EE66E010EE66EE66EE66AE66AC7
:103BC000E66AA4C7E6FFA5C7E6FFA6C7E6FFA7C744
:103BD000E6FF13EC13F0146E0C0EE15E145006C0F9
:103BE000A4F707C0A5F708C0A6F709C0A7F7010EFC
:103BF000E66EE1EC00F0E5520C0EE66EE66AE3ECF0
:103C000006F0E552E552020EE66EE1EC00F0E552F8
:103C1000A4C706F0A5C707F0A6C708F0A7C709F014
:103C20002CEC26F007C080F708C081F709C082F7A6
:103C30000AC083F70901D60E266F080E276F010E02
:103C4000E66E26C9E6FF27C9E6FF80C7E6FF81C703
:103C5000E6FF82C7E6FF83C7E6FF78EC08F0146E44
:103C6000070EE15E145026C9E6FF27C9E6FFA3EC64
:103C700000F0E552E552200EE66E61EC00F0E552F0
:103C8000480EE66E61EC00F0E5527A0EE66E61ECED
:103C900000F0E552000EE66EE66A80C7E6FF81C7D7
:103CA000E6FF82C7E6FF83C7E6FF79EC03F0146EF8
:103CB000060EE15E14500701C49F0901D60E266F5F
:103CC000080E276F010EE66E26C9E6FF27C9E6FF3C
:103CD00080C7E6FF81C7E6FF82C7E6FF83C7E6FF2E
:103CE00078EC08F0146E070EE15E145026C9E6FF6A
:103CF00027C9E6FFADEC05F0E552E552F3CF16F724
:103D0000F4CF17F7F4EC05F00701C48F200EE66E30
:103D10004E0EE66EE66AE66A1FEC0DF0E552E552DD
:103D2000E552E55200D00701C48F010EE66EE1ECCA
:103D300000F0E5520B0E070191AF02D0D89003D0EE
:103D4000905D000E915917E290C7E6FF91C7E6FF1C
:103D5000E3EC06F0E552E55239C9E6FF3AC9E6FF61
:103D60003BC9E6FF3CC9E6FFE4EC0EF0E552E55244
:103D7000E552E5523FD00B0EE66EE66AE3EC06F044
:103D8000E552E552020EE66EE1EC00F0E552050E5A
:103D9000E66E020EE66EC4EC00F0E552E552010E4E
:103DA000E66E26C9E6FF27C9E6FF80C7E6FF81C7A2
:103DB000E6FF82C7E6FF83C7E6FF78EC08F0146EE3
:103DC000070EE15E145026C9E6FF27C9E6FFA3EC03
:103DD00000F0E552E552200EE66E61EC00F0E5528F
:103DE000480EE66E61EC00F0E5527A0EE66E61EC8C
:103DF00000F0E5520701116B146B156B010E92195F
:103E000001E1935103E1926B936BA19C010E941914
:103E100001E1955103E1946B956BA19AA08CA08A66
:103E20009E909D8AC49F040EE15C02E2E16AE55225
:103E3000E16EE552E7CFD9FF1200980EE66E3A0E1A
:103E4000E66EE66AE66A1FEC0DF0E552E552E552D1
:103E5000E552E0EC0DF089980701CA6BCB6BC66B9D
:103E6000C76B600E046F000E056F04C702F705C72D
:103E700003F70901D60E266F080E276F0701B86BEE
:103E8000B96BBA6BBB6B560EC06FC16BC26BC36BA9
:103E9000010E866F876BC56BC58DC589C595C59BA2
:103EA000C591C5930F6B106B0D6B0E6BD26BD36B03
:103EB000C49F64EC05F00C0EE66EE4EC05F0E552F0
:103EC000400EE66E0D0EE66E030EE66EE66A1FEC21
:103ED0000DF0E552E552E552E552F4EC05F0E2C78B
:103EE00014F0E3C715F0166A14C0E6FF15C0E6FF2C
:103EF00016C0E6FFD60EE66E080EE66E38EC32F01F
:103F0000176E050EE15E1750D60EE66E080EE66ED1
:103F1000ADEC05F0E552E552F3CF16F7F4CF17F705
:103F2000F4EC05F0FAC714F0FBC715F0166A14C0DC
:103F3000E6FF15C0E6FF16C0E6FFD60EE66E080ED9
:103F4000E66E38EC32F0176E050EE15E1750D60EB5
:103F5000E66E080EE66EADEC05F0E552E552F3CFE5
:103F600016F7F4CF17F7F4EC05F0F6C714F0F7C71F
:103F700015F0166A14C0E6FF15C0E6FF16C0E6FF8E
:103F8000D60EE66E080EE66E38EC32F0176E050EB1
:103F9000E15E1750D60EE66E080EE66EADEC05F04B
:103FA000E552E552F3CF16F7F4CF17F7F8C714F040
:103FB000F9C715F0166A14C0E6FF15C0E6FF16C073
:103FC000E6FFD60EE66E080EE66E38EC32F0176E9F
:103FD000050EE15E1750D60EE66E080EE66EADECED
:103FE00005F0E552E552F3CF16F7F4CF17F7000EC0
:103FF000E66EE66AE3EC06F0E552E5520E0EE66E7A
:10400000E66AE3EC06F0E552E5520F0EE66EE66A6C
:10401000E3EC06F0E552E552F4EC05F0F4C714F0D9
:10402000F5C715F0166A14C0E6FF15C0E6FF16C006
:10403000E6FFD60EE66E080EE66E38EC32F0176E2E
:10404000050EE15E1750D60EE66E080EE66EADEC7C
:1040500005F0E552E552F3CF16F7F4CF17F7FC0E53
:10406000F66E560EF76E0900F5CF68F70900F5CF2A
:1040700069F70900F5CF6AF70800F5CF6BF7060E70
:10408000E66E26C9E6FF27C9E6FF68C7E6FF69C7EF
:10409000E6FF6AC7E6FF6BC7E6FF78EC08F0146E30
:1040A000070EE15E145026C9E6FF27C9E6FFADEC16
:1040B00005F0E552E552F3CF16F7F4CF17F7F4EC1D
:1040C00005F089980701C48F0EEC00F0A00EE66E93
:1040D000860EE66E010EE66EE66A1FEC0DF0E55206
:1040E000E552E552E552E66A010EE66EC4EC00F0D8
:1040F000E552E552260EE66E660EE66E80EC00F0A6
:10410000E552E552E66A020EE66EC4EC00F0E552B6
:10411000E552000EE66EE66AE3EC06F0E552E55283
:10412000900EE66ED00EE66E030EE66EE66A1FECAB
:104130000DF0E552E552E552E5520701C49F0D0E20
:10414000E66EE66AE3EC06F0E552E55278EC0DF037
:10415000FFEC0DF00701D06BD16B126B136B000EEF
:10416000125D010E135946E2FC0E1225F66E520E38
:104170001321F76E0800F5CF18F018C009F006EC0F
:1041800026F007C014F008C015F009C016F00AC0E8
:1041900017F00C6A0D6A0E6A410E0F6E14C007F01C
:1041A00015C008F016C009F017C00AF0DEEC26F0C2
:1041B00007C070F708C071F709C072F70AC073F73B
:1041C00070C707F071C708F072C709F073C70AF02B
:1041D000C4EC27F00950E66E000E07011225E96EC7
:1041E000060E1321EA6EE552E750EF6E122B000E19
:1041F0001323B5D7010E906F916B0A0E1C6F1D6BC8
:104200000901E80E396F030E3A6F3B6B3C6BF2C746
:1042100014F0F3C715F0166A14C0E6FF15C0E6FFE8
:1042200016C0E6FFD60EE66E080EE66E38EC32F0EB
:10423000176E050EE15E1750D60EE66E080EE66E9E
:10424000ADEC05F0E552E552F3CF16F7F4CF17F7D2
:104250000701B86BB96BBA6BBB6B39C906F03AC9C9
:1042600007F03BC908F03CC909F02EEC26F007C066
:1042700064F708C065F709C066F70AC067F768C742
:104280000CF069C70DF06AC70EF06BC70FF064C77A
:1042900007F065C708F066C709F067C70AF0DEECEB
:1042A00026F007C060F708C061F709C062F70AC0CE
:1042B00063F760C7E6FF61C7E6FF62C7E6FF63C753
:1042C000E6FF28EC31F0E552E552E552E55206C032
:1042D00014F007C015F008C016F009C017F014C09C
:1042E00007F015C008F016C009F017C00AF01AEC64
:1042F00028F006C0BCF707C0BDF708C0BEF709C06C
:10430000BFF7D60EE66E080EE66EBCC7E6FFBDC769
:10431000E6FFBEC7E6FFBFC7E6FF07EC2EF0146E50
:10432000060EE15E1450D60EE66E080EE66EADEC9B
:1043300005F0E552E552F3CF16F7F4CF17F7090E63
:10434000E66EE4EC05F0E552100EE66E270EE66E22
:10435000E66AE66A1FEC0DF0E552E552E552E552D9
:1043600007011E6B020E1F6FC48F010EE66EE1EC9B
:1043700000F0E552010EE66EE66AE3EC06F0E55267
:10438000E552020EE66EE1EC00F0E552D60EE66E66
:10439000080EE66EA3EC00F0E552E55239C9E6FFDF
:1043A0003AC9E6FF3BC9E6FF3CC9E6FFE4EC0EF084
:1043B000E552E552E552E5520701C49F770E7C6F46
:1043C000CC0E7D6FAB0E7E6F420E7F6F0B0EE66ED6
:1043D000E66AE3EC06F0E552E552ECC714F0EDC7EF
:1043E00015F0166A14C0E6FF15C0E6FF16C0E6FF1A
:1043F000D60EE66E080EE66E38EC32F0176E050E3D
:10440000E15E1750D60EE66E080EE66EADEC05F0D6
:10441000E552E552F3CF16F7F4CF17F7080EE66E24
:1044200026C9E6FF27C9E6FF7CC7E6FF7DC7E6FF92
:104430007EC7E6FF7FC7E6FF78EC08F0146E070E34
:10444000E15E145026C9E6FF27C9E6FFADEC05F092
:10445000E552E552F3CF16F7F4CF17F7F4EC05F079
:104460000DEC03F00C0EE66EE66AE3EC06F0E552A6
:10447000E5520701806B816BFA0E826F440E836FE9
:10448000000EE66EE66A80C7E6FF81C7E6FF82C7D8
:10449000E6FF83C7E6FF79EC03F0146E060EE15EDB
:1044A0001450010EE66E26C9E6FF27C9E6FF80C755
:1044B000E6FF81C7E6FF82C7E6FF83C7E6FF78EC29
:1044C00008F0146E070EE15E145026C9E6FF27C9F6
:1044D000E6FFADEC05F0E552E552F3CF16F7F4CF69
:1044E00017F7F4EC05F00701C49FCAEC0DF0EAC71A
:1044F00014F0EBC715F0166A14C0E6FF15C0E6FF0E
:1045000016C0E6FFD60EE66E080EE66E38EC32F008
:10451000176E050EE15E175026C9E6FF27C9E6FFB4
:10452000ADEC05F0E552E552F3CF16F7F4CF17F7EF
:10453000000EE66EE66A0DEC0EF0E552E552F3CFA2
:1045400096F7F4CF97F726C9E6FF27C9E6FF96C787
:10455000E6FF97C7E6FF6DEC2DF0E552E552E55218
:10456000E552090EE66EE4EC05F0E552560EE66EF5
:10457000E4EC05F0E5523D0EE66EE4EC05F0E552A4
:10458000200EE66EE4EC05F0E55226C9E6FF27C9E9
:10459000E6FFADEC05F0E552E552F3CF16F7F4CFA8
:1045A00017F7010EE66EE66A0DEC0EF0E552E552E5
:1045B000F3CF98F7F4CF99F726C9E6FF27C9E6FFAE
:1045C00098C7E6FF99C7E6FF6DEC2DF0E552E5527E
:1045D000E552E552090EE66EE4EC05F0E552480EB0
:1045E000E66EE4EC05F0E5523D0EE66EE4EC05F017
:1045F000E552200EE66EE4EC05F0E55226C9E6FF32
:1046000027C9E6FFADEC05F0E552E552F3CF16F70A
:10461000F4CF17F7F4EC05F00701C66BC76BC86B56
:10462000C96B47EC0EF00701146B156BA19CA19AA6
:104630009D90AB889D8AF28CF28EF28CCD90A08CEE
:10464000A08A8988D66A000EE66EE66A9AEC32F095
:10465000E552E552840ED56EF29A9D6AA06AA36A6D
:104660000701926B936B946B956BA19AA08AA19CA6
:10467000A08CD09CD08EAB889D8AF298F28CF28E62
:10468000F28CC595C49FCE6BCF6B116B0451021990
:1046900002E10551031901E1C5D0FDEC05F0070168
:1046A000076FCE2B000ECF23C49F0751580A01E19C
:1046B000A1D0190A01E18DD0130A71E0160A55E064
:1046C000100A39E0170A1DE0100A01E0ABD0010E14
:1046D000906F916B08EC10F039C9E6FF3AC9E6FF1C
:1046E0003BC9E6FF3CC9E6FFE4EC0EF0E552E552BB
:1046F000E552E552050E07018E6F8F6BFAEC0FF055
:1047000091D0020E906F916B66EC10F039C9E6FF04
:104710003AC9E6FF3BC9E6FF3CC9E6FFE4EC0EF010
:10472000E552E552E552E552050E07018E6F8F6B9B
:10473000FAEC0FF077D0030E906F916B9DEC10F0B8
:1047400039C9E6FF3AC9E6FF3BC9E6FF3CC9E6FFC7
:10475000E4EC0EF0E552E552E552E552050E070194
:104760008E6F8F6BFAEC0FF05DD0040E906F916B33
:1047700046EC11F039C9E6FF3AC9E6FF3BC9E6FF4E
:104780003CC9E6FFE4EC0EF0E552E552E552E55295
:10479000050E07018E6F8F6BFAEC0FF043D0050EFC
:1047A000906F916B9DEC11F039C9E6FF3AC9E6FFB5
:1047B0003BC9E6FF3CC9E6FFE4EC0EF0E552E552EA
:1047C000E552E552050E07018E6F8F6BFAEC0FF084
:1047D00029D00B0E906F916B0C0EE66EE66AE3EC3F
:1047E00006F0E552E552FAEC0FF0080E07018E6F65
:1047F0008F6B18D0060E906F916BC48FE66EE66AD1
:10480000E3EC06F0E552E5520701C49F060EE66EA2
:10481000E66AE3EC06F0E552E552040E07018E6FFE
:104820008F6B00D00701CE518E5DCF518F5901E3C0
:1048300084D10D0E075D01E080D1D06BD16B126B7E
:10484000136B8E51125D8F51135918E2600E1225B1
:10485000E96E000E1321EA6EEF50E66EE66AE3ECB5
:1048600032F0E552E5520701D051F324D06FD15117
:10487000F420D16F122B000E1323E3D78E51D019E1
:1048800002E18F51D1192FE0F0C714F0F1C715F0F4
:10489000166A14C0E6FF15C0E6FF16C0E6FFD60E86
:1048A000E66E080EE66E38EC32F0176E050EE15E2D
:1048B0001750D60EE66E080EE66EADEC05F0E5522A
:1048C000E552F3CF16F7F4CF17F78998200EE66E6E
:1048D0004E0EE66EE66AE66A1FEC0DF0E552E55212
:1048E000E552E55227D10B0E901901E1915169E093
:1048F000060E901901E1915143E0010E901901E17A
:10490000915115E0020E901901E1915110E0030E52
:10491000901901E191510BE0040E901901E19151C0
:1049200006E0050E901901E1915101E003D1BC6B45
:10493000BD6BBE6BBF6B0001656B600EE66E000E5B
:10494000E66EC2EC2CF0E552E55206C039F907C01C
:104950003AF908C03BF909C03CF939C9E6FF3AC940
:10496000E6FF3BC9E6FF3CC9E6FFE4EC0EF0E5528A
:10497000E552E552E552090E0701906F916BDAD0CE
:104980000001646B600EE66E000EE66E4DEC2CF0DE
:10499000E552E552F3CF16F7F4CF17F70701FE0EF5
:1049A000165D030E17590CE2020ED8801655000E44
:1049B000175506E216C71EF717C71FF7FDEC11F0D3
:1049C000B9D00001686B600EE66E000EE66EC2ECB8
:1049D0002CF0E552E55206C0A4F707C0A5F708C0C1
:1049E000A6F709C0A7F7A4C706F0A5C707F0A6C792
:1049F00008F0A7C709F02CEC26F007C080F708C024
:104A000081F709C082F70AC083F7000EE66EE66AF6
:104A100080C7E6FF81C7E6FF82C7E6FF83C7E6FFE0
:104A200079EC03F0146E060EE15E14500701C48F9A
:104A3000020EE66EE1EC00F0E552030EE66E020EA9
:104A4000E66EC4EC00F0E552E552010EE66E26C9B2
:104A5000E6FF27C9E6FF80C7E6FF81C7E6FF82C7FA
:104A6000E6FF83C7E6FF78EC08F0146E070EE15E00
:104A7000145026C9E6FF27C9E6FF51EC32F0E55293
:104A8000E552F3CF14F7F4CF15F707010A0ED880DB
:104A90001457000E1557070114C714F015C715F069
:104AA0001407000E155BD8801454000E155406E24E
:104AB000200EE66E61EC00F0E552EDD726C9E6FF68
:104AC00027C9E6FFA3EC00F0E552E552200EE66EA2
:104AD00061EC00F0E552480EE66E61EC00F0E55244
:104AE0007A0EE66E61EC00F0E5520701C49F010EFC
:104AF000E66E26C9E6FF27C9E6FF80C7E6FF81C745
:104B0000E6FF82C7E6FF83C7E6FF78EC08F0146E85
:104B1000070EE15E145026C9E6FF27C9E6FFADEC9B
:104B200005F0E552E552F3CF16F7F4CF17F7F4ECA2
:104B300005F000D08988FAEC0FF00701103504E287
:104B40000F510008000E105507E30E3504E20D5119
:104B50000008000E0E5529E2E0C7E6FFE1C7E6FFB8
:104B600074EC05F0E552E552F3CF0BF7F4CF0CF7F8
:104B7000E66A0FC7E6FF10C7E6FF7EEC07F0E552D6
:104B8000E552E552090EE66EE4EC05F0E552E66A00
:104B90000DC7E6FF0EC7E6FF7EEC07F0E552E552D3
:104BA000E5528998FAEC0FF001D089880701C48F8B
:104BB000010EE66EE1EC00F0E55290C7E6FF91C70A
:104BC000E6FFE3EC06F0E552E5520701C49F9E9034
:104BD000146B156BBA51EA6A000FE96E060EEA22F1
:104BE000EFCF40FFBC0EE96E070EEA6EB851EE241F
:104BF000B86FB951EE20B96FBA51EE20BA6FBB5100
:104C0000EE20BB6F1151E6E041D51200019E05D0A8
:104C1000019E09AE02D0096C018E09C003F0026A40
:104C2000136A126A860E046E056AD4EF28F0019E9C
:104C300008D0019E09AE05D0086C091EE86A092259
:104C4000018E09C003F008C002F0136A126A8E0ECA
:104C5000046E056AD4EF28F0019E0CD0019E09AEC7
:104C600009D0066C071E081E091EE86A07220822E2
:104C70000922018E09C003F008C002F007C013F03A
:104C800006C012F09E0E046E056AD4EF28F00F7E67
:104C9000016A10EC29F028EC29F001B6B8EF28F0F1
:104CA00001A20AD001AA03D001BEB8EF28F001A4E6
:104CB000C4EF28F0C1EF28F001AA05D001ACC4EF81
:104CC00028F0C1EF28F001A00AD001A808D001BE49
:104CD00004D001A402D0CDEF28F0D1EF28F0126A61
:104CE000056A0F500A5C116E10E307C013F008C08C
:104CF00002F009C003F00AC010F00CC007F00DC0AC
:104D000008F00EC009F0013A09D00CC013F00DC034
:104D100002F00EC003F00FC010F0116C019E01BC38
:104D2000018E10C004F001B000EF29F01A0E1160DE
:104D300000EF29F0046A0A6A01A408D0076C081E73
:104D4000091E0A1EE86A082209220A2201AC08D0BC
:104D5000136C021E031E041EE86A022203220422B0
:104D6000066A115207E00A34093208320732063265
:104D7000112EF9D70750132608500222095003229A
:104D80000A50042206C012F0019E04AE0BD0126C31
:104D9000131E021E031E041EE86A132202220322AF
:104DA0000422018E04A006D0D880033202321332CE
:104DB0001232102A10C004F0D4EF28F0016A10EC6F
:104DC00029F028EC29F001B6B8EF28F001A205D0AF
:104DD00001BAB8EF28F0BFEF28F001BACBEF28F006
:104DE00001A005D001B8B8EF28F0CBEF28F001B84A
:104DF000BFEF28F0056A7F0E0A24046EE86A0522D8
:104E00000F50045EE86A055A1A0E106E0A6A126A9A
:104E1000136A026A036A0C50075E0D50085A0E505E
:104E2000095A000E0A5A09E70C5007260D500822AD
:104E30000E500922000E0A2201D0128AD89007369D
:104E4000083609360A36D89012361336023603363B
:104E5000102EE1D7095008100710D8A4128AD4EFF9
:104E600028F0016A10EC29F028EC29F001B6B8EF1F
:104E700028F001A205D001B8B8EF28F0BFEF28F064
:104E800001AA05D001B0B8EF28F0BFEF28F001B0BB
:104E900002D001A802D0CBEF28F0056A0F500A24F7
:104EA000046EE86A05227E0E045EE86A055A126AFC
:104EB000136A026A036A0E500902F4CF03F0F3CFBB
:104EC00002F00D500902F3501326F4500222000E96
:104ED00003220E500802F3501326F4500222000E53
:104EE00003220C500902F3501226F4501322000E34
:104EF000022203220D500802F3501226F45013220E
:104F0000000E022203220E500702F3501226F45024
:104F10001322000E022203220C500802F450122623
:104F2000000E1322022203220D500702F450122613
:104F3000000E132202220322D4EF28F0006A0EAEE4
:104F4000A7EF27F00D6C0E1EE86A0E22001E09AEB8
:104F5000AFEF27F0086C091EE86A0922001ECDECAD
:104F600032F009BEBFEF27F000AE000C086C091E3E
:104F7000E86A0922046C051EE86A0522000C00BEDE
:104F8000B6EF27F00188FF0C016A10EC29F001B69A
:104F9000CEEF27F001A20AD001B403D07F0E096E34
:104FA00019D0800E096E16D0096A14D001B0FCD752
:104FB000870E0A60F1D77E0E0A64F6D7860E0A5C69
:104FC00004E0D89009320A2AF9D701A403D0096C69
:104FD00009AEEAD71200016A10EC29F001B6F5EF2C
:104FE00027F001A20ED001B405D07F0E096EFF0E8E
:104FF000086E1FD0800E096E086A1BD0096A086A05
:1050000018D001B0FBD78F0E0A60EDD77E0E0A6470
:10501000F5D78E0E0A5C05E0D890093208320A2ACC
:10502000F8D701A406D0086C091EE86A092209AE67
:10503000E5D71200016A10EC29F001B624EF28F040
:1050400001A20FD001B407D07F0E096EFF0E086ECB
:10505000076E066E25D0800E096E01D0096A000E1B
:10506000F6D701B0FBD7066A9F0E0A60EBD77E0E1B
:105070000A64F4D79E0E0A5C07E0D8900932083221
:10508000073206320A2AF6D701A40AD0066C071E98
:10509000081E091EE86A07220822092209AEDED787
:1050A000120063EC28F001B6000C01B0000C01B452
:1050B000000C010C63EC28F001B6000C01B0000CF0
:1050C00001A4000C010C016A10EC29F028EC29F075
:1050D00001B6120001AE08D001A004D001A802D090
:1050E00001801200019012000F500A5C0BE10E507B
:1050F000095C08E10D50085C05E10C50075C02E119
:1051000001801200D8A002D0018E10D00A500FC02A
:105110000AF00F6E09500EC009F00E6E08500DC057
:1051200008F00D6E07500CC007F00C6E0F500A5CB3
:1051300010E0FF0F09E0019001B403D001AE01843B
:10514000120001AE019412000F2AD8900E320D32D7
:105150000C320C50075E0D50085A0E50095A09BE09
:10516000EAD7D8900736083609360A2EF8D7C8D7B6
:105170007F0E0A6EFF0E096E086E076E12007F0E1C
:1051800001BEFF0E0A6E02D07F0E0A6E800E096EFF
:10519000086A076AF3D701AE04D0800E0A6E096A66
:1051A000F7D70A6A096AF4D70350021013101210D5
:1051B000F8E005BEF0D703BE0CD004500510EBE0BC
:1051C000D89012361336023603360406D8A00506E8
:1051D000F2D70550D4E10428D2E012AE11D07F0EF0
:1051E000121402E113A00CD0132AE86A022203224F
:1051F00007E3D880033202321332042A0428BFE0C6
:105200000450C9E013C007F002C008F00334096E6F
:1052100004300A6E09320A9E01BE0A8EBEEF28F0E3
:1052200009360A3602E30184017E06E101800A6A3A
:10523000096A086A076A12000A2803E0D88009325E
:105240001200D890093202E1018212000186120098
:105250000E360F3602E3018C017E06E101880F6AEB
:105260000E6A0D6A0C6A12000F2803E0D8800E3215
:105270001200D8900E32EAE1018A1200008080808C
:105280008080800000C0C0C0C0C0C00000E0E0E07E
:10529000E0E0E00000F0F0F0F0F0F00000F8F8F8E6
:1052A000F8F8F80000FCFCFCFCFCFC0000FEFEFE34
:1052B000FEFEFE0000FFFFFFFFFFFF000010181CB6
:1052C0001E1C1810000103070F070301040E1F0E18
:1052D0000E0E0E0E0E0E0E0E0E1F0E0402040E11FA
:1052E0001F100E0008040E111F100E0008040E01FE
:1052F0000F110F0002050200000000008082858867
:105300008B8E9194979A9DA0A2A5A8ABADB0B3B592
:10531000B8BBBDC0C2C5C7C9CCCED0D2D4D6D8DAEE
:10532000DCDEE0E2E3E5E6E8E9EBECEDEEEFF0F100
:10533000F2F3F4F5F5F6F6F7F7F7F7F7F8F7F7F70E
:10534000F7F7F6F6F5F5F4F3F2F1F0EFEEEDECEB3E
:10535000E9E8E6E5E3E2E0DEDCDAD8D6D4D2D0CE86
:10536000CCC9C7C5C2C0BDBBB8B5B3B0ADABA8A5AD
:10537000A2A09D9A9794918E8B888582807D7A7762
:1053800074716E6B6865625F5D5A5754524F4C4A38
:105390004744423F3D3A383633312F2D2B292725BC
:1053A00023211F1D1C1A19171614131211100F0E8A
:1053B0000D0C0B0A0A09090808080808080808085B
:1053C000080809090A0A0B0C0D0E0F10111213140C
:1053D0001617191A1C1D1F21232527292B2D2F31A4
:1053E0003336383A3D3F4244474A4C4F5254575A5D
:1053F0005D5F6265686B6E7174777A7D0001020390
:105400000405060708090A0B0C0D0E0F10111213E4
:105410001415161718191A1B1C1D1E1F20212223D4
:105420002425262728292A2B2C2D2E2F30313233C4
:105430003435363738393A3B3C3D3E3F40414243B4
:105440004445464748494A4B4C4D4E4F50515253A4
:105450005455565758595A5B5C5D5E5F6061626394
:105460006465666768696A6B6C6D6E6F7071727384
:105470007475767778797A7B7C7D7E7F8081828374
:105480008485868788898A8B8C8D8E8F9091929364
:105490009495969798999A9B9C9D9E9FA0A1A2A354
:1054A000A4A5A6A7A8A9AAABACADAEAFB0B1B2B344
:1054B000B4B5B6B7B8B9BABBBCBDBEBFC0C1C2C334
:1054C000C4C5C6C7C8C9CACBCCCDCECFD0D1D2D324
:1054D000D4D5D6D7D8D9DADBDCDDDEDFE0E1E2E314
:1054E000E4E5E6E7E8E9EAEBECEDEEEFF0F1F2F304
:1054F000F4F5F6F7F8F9FAFBFCFDFEFFFFFFFFFFFE
:10550000FFFFFFFFFFFFFFFFFFFFFFFFFFFFFFFFAB
:10551000FFFFFFFFFFFFFFFFFFFFFFFFFFFFFFFF9B
:10552000FFFFFFFFFFFFFFFFFFFFFFFFFFFFFFFF8B
:10553000FFFFFFFFFFFFFFFFFFFFFFFFFFFFFFFF7B
:10554000FFFFFFFFFFFFFFFFFFFFFFFFFFFFFFFF6B
:10555000FFFFFFFFFFFFFFFFFFFFFFFFFFFFFFFF5B
:10556000FFFFFFFFFFFFFFFFFFFFFFFFFFFFFFFF4B
:10557000FFFFFFFFFFFFFFFFFFFFFFFF0000000037
:10558000000000000000000000000000000000001B
:10559000000000000000000000000000000000000B
:1055A00000000000000000000000000000000000FB
:1055B00000000000000000000000000000000000EB
:1055C00000000000000000000000000000000000DB
:1055D00000000000000000000000000000000000CB
:1055E00000000000000000000000000000000000BB
:1055F00000000000000000000000000008090B0D82
:105600000F11131517181A1C1E2022242627292BC8
:105610002D2F31333536383A3C3E404244454749D8
:105620004B4D4F51535456585A5C5E6062636567E8
:10563000696B6D6F71727476787A7C7E80818385F8
:1056400087898B8D8F90929496989A9C9E9FA1A308
:10565000A5A7A9ABADAEB0B2B4B6B8BABCBDBFC118
:10566000C3C5C7C9CBCCCED0D2D4D6D8DADBDDDF28
:10567000E1E3E5E7E9EAECEEF0F2F4F6F8F6F4F24D
:10568000F0EEECEAE9E7E5E3E1DFDDDBDAD8D6D4FA
:10569000D2D0CECCCBC9C7C5C3C1BFBDBCBAB8B6CA
:1056A000B4B2B0AEADABA9A7A5A3A19F9E9C9A989A
:1056B000969492908F8D8B8987858381807E7C7A6A
:1056C00078767472716F6D6B6967656362605E5C3A
:1056D0005A58565453514F4D4B4947454442403E0A
:1056E0003C3A38363533312F2D2B292726242220DA
:1056F0001E1C1A18171513110F0D0B094CD8B43CAA
:105700004672616D65204572726575722065742000
:105710004F766572666C6F77206465746563746933
:105720006F6E203A2000506F727420636F6D6D2091
:105730003338343030626473206F7576657274006C
:105740004D61727175657220322520647520736910
:10575000676E616C0045534320706F757220736FE4
:10576000727469720D0043617074757265205461C2
:105770007578207375722041444330200020496EB3
:10578000697420436F6D70617261746F7273203140
:105790002065742032203A200020466163746575CC
:1057A000722044445320414439383335203D200091
:1057B00020557361676520513D31304D687A2078FE
:1057C0003428504C4C290D002045727265757220AA
:1057D0005361697369652E2E2E2E2E0D0020496EA1
:1057E000697420436F6E734672657120314B687A1D
:1057F0000900204661637465757220444453203D5E
:10580000200020496E746572666163652076696167
:10581000205465726D696E616C20525332333220B0
:1058200045542F4F552076696120436C6176696538
:1058300072203520746F7563686573202B204C438C
:10584000440D002047616D6D652064652031206145
:105850002032352E303030487A20200D002031386B
:105860004634364B32325F4444535F313330343147
:10587000325F41444335625F4144393833355F4CD0
:1058800043445F52533233325F4A6F7973746963B2
:105890006B5F4331382E630D00FFFF0EE3CFEAFF4D
:1058A000E552FF0EE3CFE9FFE552E66AE66AD9CF9B
:1058B000E6FFDACFE6FFFC0EE124D96EFF0EE22010
:1058C000DA6EE66AE66AE66A200EEF5C06E0090E2A
:1058D000EF5C03E0EF6603D03FD0EE50F5D72D0E1E
:1058E000EF5C03E1FF0EE32A03D02B0EEF5C01E136
:1058F000EE502F0EEF6424D03A0EEF6021D0D890F6
:10590000F90EE336FA0EE336FD0EDECFE3FFFE0EB0
:10591000DDCFE3FFD890F90EE336FA0EE336D890E8
:10592000F90EE336FA0EE336FD0EE350DE26FE0EE8
:10593000E350DD22300EEE5CDE26000EDD22D9D7EC
:10594000FF0EE3CFE8FFE85207E0F90EE31EE32A7B
:10595000FA0ED8B4E306E31EE552E552E552FF0E17
:10596000E3CFDAFFE552FF0EE3CFD9FFE552E1CFF7
:10597000E9FFE2CFEAFFED52ED52EECFF3FFEFCFBA
:10598000F4FF1200FF0EE3CFEAFFE552FF0EE3CF74
:10599000E9FFE552E66AE66AE66AE66AD9CFE6FF1B
:1059A000DACFE6FFFA0EE124D96EFF0EE220DA6EBE
:1059B000E66AE66AE66AE66AE66A200EEF5C06E0F8
:1059C000090EEF5C03E0EF6603D06BD0EE50F5D725
:1059D0002D0EEF5C03E1FF0EE32A03D02B0EEF5CEC
:1059E00001E1EE502F0EEF6444D03A0EEF6041D04B
:1059F000D890F50EE336F60EE336F70EE336F80EE2
:105A0000E336FB0EDECFE3FFFC0EDECFE3FFFD0E41
:105A1000DECFE3FFFE0EDDCFE3FFDD52DD52D89097
:105A2000F50EE336F60EE336F70EE336F80EE33600
:105A3000D890F50EE336F60EE336F70EE336F80EA1
:105A4000E336FB0EE350DE26FC0EE350DE22FD0EB5
:105A5000E350DE22FE0EE350DD22DD52DD52300E39
:105A6000EE5CDE26000EDE22DE22DD22DD52DD527D
:105A7000B9D7FF0EE3CFE8FFE85213E0F50EE31EBF
:105A8000F60EE31EF70EE31EF80EE31EF50EE32AF4
:105A900008E1F60EE32A05E1F70EE32A02E1F80E2B
:105AA000E32AE552E552E552E552E552D9CFE9FF46
:105AB000DACFEAFFEECF06F0EECF07F0EECF08F038
:105AC000EFCF09F0FF0EE3CFDAFFE552FF0EE3CF91
:105AD000D9FFE552E552E5521200D9CFE6FFDACF01
:105AE000E6FFFA0EE3CFD9FFFB0EE3CFDAFFFD0EA0
:105AF000E35209E72D0EDE6EFC0EE31EE32AFD0ED7
:105B0000D8B4E306E31EE652E652E652FD0EE12467
:105B1000E76EFF0EE220E46EE652F70EE3CFE6FFFB
:105B2000F70EE3CFE6FFDDEC2DF0F90EE124E96E90
:105B3000FF0EE220EA6ECDEC2DF00AE1CAEC2DF06A
:105B400009E1CDEC2DF008E1CAEC2DF007E108D019
:105B5000D8EC2DF0D3EC2DF0D8EC2DF0D3EC2DF0CB
:105B6000D8EC2DF0DE6AF90EE126FF0EE222FF0EE0
:105B7000E3CFDAFFE552FF0EE3CFD9FFE552FC0E8B
:105B8000E124E96EFF0EE220EA6EEECFF3FFEFCFE5
:105B9000F4FF1200EF380F0B1200EF500F0B02E171
:105BA000EE52D8841200EF380F0B300FDE6E120069
:105BB000EE500F0B300FDE6E1200FC0EE3CFE9FF4C
:105BC000FD0EE3CFEAFF100EE66EEE6AEE6AEF6AB4
:105BD000D890FD0EE336FE0EE336ED36ED36EF36A9
:105BE000FF0EE30609E0FEEC2DF0EE52FEEC2DF088
:105BF000EE52FEEC2DF0EDD7E56E1200030EEF2411
:105C0000E8B6EF6E300EEF24E8BEEF6E000CD9CF91
:105C1000E6FFDACFE6FFF80EE3CFD9FFF90EE3CFC8
:105C2000DAFFE652E652E652E652E652FB0EE12475
:105C3000E76EFF0EE220E46EE652F30EE3CFE6FFDE
:105C4000F30EE3CFE6FFF30EE3CFE6FFF30EE3CF71
:105C5000E6FF8CEC2EF0F50EE124E96EFF0EE2205B
:105C6000EA6E79EC2EF019E17CEC2EF018E179EC7B
:105C70002EF017E17CEC2EF016E179EC2EF015E118
:105C80007CEC2EF014E179EC2EF013E17CEC2EF09C
:105C900012E179EC2EF011E112D082EC2EF087ECBB
:105CA0002EF082EC2EF087EC2EF082EC2EF087ECBA
:105CB0002EF082EC2EF087EC2EF082EC2EF087ECAA
:105CC0002EF0DE6AF50EE126FF0EE222FF0EE3CF94
:105CD000DAFFE552FF0EE3CFD9FFE552FA0EE124D9
:105CE000E96EFF0EE220EA6EEECFF3FFEFCFF4FF96
:105CF0001200EF380F0B1200EF500F0B02E1EE52C3
:105D0000D8841200EF380F0B300FDE6E1200EE5009
:105D10000F0B300FDE6E1200FA0EE3CFE9FFFB0E21
:105D2000E3CFEAFF200EE66EEE6AEE6AEE6AEE6AF6
:105D3000EF6AD890FB0EE336FC0EE336FD0EE33639
:105D4000FE0EE336ED36ED36ED36ED36EF36FF0E70
:105D5000E3060FE0BBEC2EF0EE52BBEC2EF0EE5261
:105D6000BBEC2EF0EE52BBEC2EF0EE52BBEC2EF064
:105D7000E1D7E56E1200030EEF24E8B6EF6E300EA9
:105D8000EF24E8BEEF6E000CD9CFE6FFDACFE6FFD6
:105D9000E1CFD9FFE2CFDAFF130EE12402E3E1689D
:105DA000E652E16E0C0EDB6AD950FA0FE96EFF0E77
:105DB000DA20EA6E080EEECFDBFF090EEECFDBFF36
:105DC0000A0EEECFDBFF0B0EEECFDBFF1FD9D95053
:105DD000080F17D9EECFE6FFEECFE6FFEECFE6FFD6
:105DE000EFCFE6FF0DEC30F0146E060EE15C02E240
:105DF000E16AE552E16E1450DF6E020EDF5C01E0F5
:105E0000BCD0050EDBCF16F0060EDBCF17F0F80E78
:105E1000DB50165C146EF90EDB501758156E7F0EB2
:105E2000145E000E155A0D0E14C0DBFF0E0E15C0C9
:105E3000DBFF0D0E0E0EDBCF15F00001800E1514EA
:105E40000AE0010EF36E0C0EF3CFDBFF070EDB5002
:105E500001E098D09DD00D0EDBCF14F00E0EDBCFFD
:105E600015F0D890155004E6170E145C000E155866
:105E700001E39ED0186819687F0E1A6E1B6A0D0E1A
:105E8000DB501F0B18C014F019C015F01AC016F023
:105E90001BC017F007E0D8901732163215321432B3
:105EA000E806F9E10F0E14C0DBFF100E15C0DBFF92
:105EB000110E16C0DBFF120E17C0DBFF0F0EDBCF7B
:105EC00014F0100EDBCF15F0110EDBCF16F0120E12
:105ED000DBCF17F0D950010F94D8EE501416EE50C6
:105EE0001516EE501616EE50171614501510161003
:105EF000171002E1000E01D0010EE76E0C0EE7CF85
:105F0000DBFFDB5055E0186A196A800E1A6E1B6AB7
:105F1000010E1C6E1D6A1E6A1F6AD9500F0F71D8C0
:105F2000EE501C26EE501D22EE501E22EE501F2277
:105F30001C50185C146E1D501958156E1E501A58BE
:105F4000166E1F501B58176ED950010F5AD8145097
:105F5000EE161550EE161650EE161750EE16D950D6
:105F6000080FE66E000EDA20E66E50D89BEC30F09B
:105F7000E552E552E552E5521BD0DF0419E1070E68
:105F8000DB5006E0146A156A166A800E176E04D09C
:105F9000146A156A166A176A080E14C0DBFF090E28
:105FA00015C0DBFF0A0E16C0DBFF0B0E17C0DBFFB0
:105FB000F60EDBCFE9FFF70EDBCFEAFF0C0EDBCFEF
:105FC000EFFF080EDBCF14F0090EDBCF15F00A0E41
:105FD000DBCF16F00B0EDBCF17F014C006F015C0A8
:105FE00007F016C008F017C009F0130EE15C02E2DA
:105FF000E16AE552E16EE552E5CFDAFFE7CFD9FF7E
:106000001200E96E000EDA20EA6E1200D950010F7C
:10601000E66E000EDA20E66E1200D9CFE6FFDACF88
:10602000E6FFE1CFD9FFE2CFDAFFE6521468156848
:106030007F0E166E176AD950FA0FE96EFF0EDA203E
:10604000EA6EEE501416EE501516EE501616EE507F
:1060500017166AD814C0EEFF15C0EEFF16C0EEFF8B
:1060600017C0EEFFFD0EDB50800B02E0010E01D0E9
:10607000000EE66E59D8060EE926000EEA22E55219
:10608000E750EF6EFC0EDBCF14F0FD0EDBCF15F00A
:10609000D89014361536FC0E14C0DBFFFD0E15C06B
:1060A000DBFFDB50E66E40D8040EE926000EEA2244
:1060B000E552E750EE6EED6AFD0EDB50146E156A88
:1060C000FF0E141818E1155016E12ED8EECF14F07B
:1060D000EECF15F0EECF16F0EFCF17F014501510ED
:1060E0001610171006E0210E0001EA6FEB6B800E10
:1060F0000BD0040E09D0FD0EDB5008E115D8EE6A76
:10610000EE6AEE6AEE6A010EDF6E06D0020EDF6EF8
:106110000BD8EE52EE52EE8EDF50E552E552E5CF4F
:10612000DAFFE7CFD9FF1200F80EDBCFE9FFF90E57
:10613000DBCFEAFF1200D9CFE6FFDACFE6FFE1CFEF
:10614000D9FFE2CFDAFF5BD8153411E21450FE0814
:10615000000E15540CE276D805E06CD8800EEE6E79
:10616000EE6847D067D8800EEE6E7F0E0ED047D80F
:10617000D890155004E6010E145C000E15580BE281
:1061800061D805E057D8EE6A800EEE6E32D052D854
:10619000EE6AEE6A2ED047D8EECF14F0EECF15F0AF
:1061A000EECF16F0EFCF17F032D814C0EEFF15C0C7
:1061B000EEFF16C0EEFF17C0EEFF21D81450010B02
:1061C00005E025D8020E3AD8EF8E04D020D8020E72
:1061D00035D8EF9E14D8D8901532143218D8030E43
:1061E0002DD814C0EFFF1AD804E011D8030E26D81A
:1061F000EF8EE552E5CFDAFFE7CFD9FF120013D8D3
:10620000040E1CD8EECF14F0EFCF15F01200FA0EEA
:10621000DBCFE9FFFB0EDBCFEAFF120004D8060E4E
:106220000DD8EF501200FC0EDBCFE9FFFD0EDBCFE7
:10623000EAFF1200ECDFEE6AEE6A1200E926000EB9
:10624000EA221200220E0001EA6FEB6B0EEF31F032
:10625000D9CFE6FFDACFE6FFE1CFD9FFE2CFDAFF11
:10626000060EE12402E3E168E652E16ED950050F23
:10627000E66E000EDA20E66E000EE66EE66AD95093
:10628000FA0FE96EFF0EDA20EA6EEECFE6FFEECFF0
:10629000E6FFEECFE6FFEFCFE6FFC4EC2EF0146E84
:1062A000080EE15C02E2E16AE552E16E1450010E73
:1062B00006C0DBFF020E07C0DBFF030E08C0DBFFDA
:1062C000040E09C0DBFF050EDB502AE0040EDB5094
:1062D000800B26E1146A156A800E166E3F0E176E4B
:1062E000D950010FE96E000EDA20EA6EEECF07F00A
:1062F000EECF08F0EECF09F0EFCF0AF014C00CF0AB
:1063000015C00DF016C00EF017C00FF048EC26F0C7
:106310000AC0EDFF09C0EDFF08C0EDFF07C0EFFFA9
:10632000010EDBCF14F0020EDBCF15F0030EDBCF36
:1063300016F0040EDBCF17F014C006F015C007F0FE
:1063400016C008F017C009F0060EE15C02E2E16A2F
:10635000E552E16EE552E5CFDAFFE7CFD9FF120053
:106360000E0EF66E000EF76E000EF86E00010900BC
:10637000F550E56F0900F550E66F03E1E56701D0E0
:106380003DD00900F550E06F0900F550E16F0900BC
:10639000F550E26F09000900F550E96E0900F5506B
:1063A000EA6E090009000900F550E36F0900F55095
:1063B000E46F09000900F6CFE7F0F7CFE8F0F8CF77
:1063C000E9F0E0C0F6FFE1C0F7FFE2C0F8FF00012E
:1063D000E35302E1E45307E00900F550EE6EE307F2
:1063E000F8E2E407F9D7E7C0F6FFE8C0F7FFE9C035
:1063F000F8FF0001E507000EE65BBFD71200D9CF1A
:10640000E6FFDACFE6FFE1CFD9FFE2CFDAFFAC6AF1
:10641000AB6AFD0EDBB0AC88DBA202D0AC8CAB8CDF
:10642000DBB4AC8EDBA602D0AB8801D0AB8ADBB884
:10643000AC84DBBAAB86DBAC02D09D8A01D09D9ADE
:10644000DBAE02D09D8801D09D98FB0EDB50AF6E75
:10645000FC0EDBCF15F015C014F0156A1450B06EA9
:10646000AC8AAB8EE552E5CFDAFFE7CFD9FF120059
:10647000FB0EE3CFF6FFFC0EE3CFF7FFFD0EE3CFFD
:10648000F8FFFE0EE3CFE9FFFF0EE3CFEAFFE9CF0F
:10649000F3FFEACFF4FF0900F5CFEFFFEE66FBD77D
:1064A0001200FE0EE3CFE9FFFF0EE3CFEAFFF36A2F
:1064B000F46AEE5203E0F34AF42AFBD71200D9CF74
:1064C000E6FFDACFE6FFE1CFD9FFE2CFDAFFE6520F
:1064D000F20E0001EC17ABAC03D0EC91ABB0EC8149
:1064E000ABB4EC85ABB2EC87AE50DF6EDF50E5525B
:1064F000E552E5CFDAFFE7CFD9FF1200D9CFE6FFAB
:10650000DACFE6FFE1CFD9FFE2CFDAFFE652E6527B
:10651000FC0EDBCFDEFFDBCFDDFF010EDB50CF6EED
:10652000DF50CE6EE552E552E552E5CFDAFFE7CF18
:10653000D9FF1200D9CFE6FFDACFE6FFE1CFD9FFCE
:10654000E2CFDAFFE652E652FC0EDBCFDEFFDBCF16
:10655000DDFF010EDB50D76EDF50D66EE552E552FF
:10656000E552E5CFDAFFE7CFD9FF1200D9CFE6FF3A
:10657000DACFE6FFE1CFD9FFE2CFDAFFACAC04D04F
:10658000AC900001ECB3AC80FD0EDB50AD6EE5527B
:10659000E5CFDAFFE7CFD9FF1200056A046A100ED3
:1065A000E76ED89008360936043605360D50045C7F
:1065B0000E50055805E30D50045E0E50055A082A8A
:1065C000E72EF0D71200F36AF46AFF0EE124E96EB9
:1065D000FF0EE220EA6EED6607D02F0EEF6404D0C6
:1065E0003A0EEF6001D0F32A1200380EF36E00EE7F
:1065F00000F00F0E01D81200EA6002D0EE6AFCD75C
:10660000F350E9601200EE6AFCD71EEE00F02EEEA9
:1066100000F0F86A019CB0EC31F003EC00F01DECE6
:106620001FF0FBD7120031384634364B323220444B
:106630004453204331380020342E3039365600FF81
:10664000FF0EE350E84E1200000000D000D000D052
:10665000E82EFAD71200C450176E166AC3501610EF
:10666000F36E17C0F4FF1200C250020B01E0010EDE
:106670001200C282120000572657405755576657DE
:106680007D579957B057C857DD57F25702584358AE
:106690005D580100020005000A0014003200640089
:1066A000C800F401EE02E803E204DC05D606D007D8
:1066B000C409BE0AB80BAC0DA00F941188137C1549
:1066C00070176419581B4C1D401F342128231C25AA
:1066D0001027F82AE02EC832B036983A803E684239
:1066E0005046384A204E0852F055D859C05DA8612E
:1066F00090657869606D487130751879007DE88023
:10670000D084B888A08C889070945898409C04A637
:10671000C8AF0000010002000A0019003200640046
:10672000FA00F401EE02E803000001000200050097
:106730000A0032006400FA00F401E8038813000044
:10674000000001000000050000000A000000320007
:10675000000064000000F4010000E803000088135A
:10676000000010270000A0860100FC5250524F4A42
:1067700045543A2031384634364B32325F44445324
:106780005F4144393833352E6D63700009090909BA
:106790000909090909090909090909090909090969
:1067A0000909090909090909090909090909090959
:1067B000090909090909090909090909D60831322C
:1067C0003334353637383930313233343500000020
:1067D0000000000000000000000000FFFFFFFFFFBE
:1067E000FFFFFFFFFFFFFFFFFFFFFFFFFFFFFFFFB9
:1067F000FFFFFFFFFFFFFFFFFFFFFFFFFFFFFFFFA9
:10680000FFFFFFFFFFFFFFFFFFFFFFFFFFFFFFFF98
:10681000FFFFFFFFFFFFFFFFFFFFFFFFFFFFFFFF88
:0200000400F00A
:100000002031384634364B32322034304D687A2035
:10001000513D31304D687A20504C4C78340D000001
:100020002053696E7573202020202020202020205E
:10003000202020202020202020202020200D000013
:100040002043617272652020202020202020202063
:10005000202020202020202020202020200D0000F3
:1000600020547269616E676C65202020202020205A
:10007000202020202020202020202020200D0000D3
:100080002044656E742064652073636965202020B8
:10009000202020202020202020202020200D0000B3
:1000A00020526576657273652064656E74206465A0
:1000B000207363696520202020202020200D00006F
:1000C0002052656374616E676C65206628546175A3
:1000D000782920202020202020202020200D000012
:1000E000205265676C6167652054617578205265A0
:1000F0006374616E676C652028706F74290D000051
:10010000205265676C616765206D61786920736F47
:10011000727469652044414320566F6C740D000071
:100120002043686F697820467265712E50494344B8
:1001300044532031207061726D692036330D000008
:10014000205265676C6167652046696E204672655E
:100150007175656E6365205049434444530D00003A
:100160002047657374696F6E2044445320414439BD
:100170003833352053504920736F6674770D000073
:10018000205265676C616765204672657120444442
:1001900053204144393833352061203A2020000073
:1001A00020496E697420736F7274696520444143FD
:1001B000206D6178692061203A20202020200000F5
:1001C000204D504C4142204944452056382E39306C
:1001D0002C4331382056332E34342E20200D00008D
:1001E0002056657273696F6E2031322F30342F3193
:1001F0003320207061756C666A756A6F200D00008F
:1002000056657273696F6E2031322F30342F31335F
:10021000202020202053494E5553202020202020EC
:100220002020202020436172726520202020202081
:100230002020202020547269616E676C6520202088
:100240002044656E74732064652053434945202023
:100250007265762044656E74206465205343494579
:100260002020202052656374616E676C6520202019
:100270005265676C2E544155582052656374616E07
:10028000202020202020202020202020202020206E
:1002900043686F6978204672657120466978657396
:1002A0005265676C2E467265712050494344445331
:1002B0004D6F646520444453202041443938333520
:1002C0005265676C2E46726571204144393833356A
:1002D000202020202020202020202020202020201E
:1002E0004630206F7520463120204144393833355F
:1002F00020202020202020202020202020202020FE
:10030000FFFFFFFFFFFFFFFFFFFFFFFFFFFFFFFFFD
:10031000FFFFFFFFFFFFFFFFFFFFFFFFFFFFFFFFED
:10032000FFFFFFFFFFFFFFFFFFFFFFFFFFFFFFFFDD
:10033000FFFFFFFFFFFFFFFFFFFFFFFFFFFFFFFFCD
:10034000FFFFFFFFFFFFFFFFFFFFFFFFFFFFFFFFBD
:10035000FFFFFFFFFFFFFFFFFFFFFFFFFFFFFFFFAD
:10036000FFFFFFFFFFFFFFFFFFFFFFFFFFFFFFFF9D
:10037000FFFFFFFFFFFFFFFFFFFFFFFFFFFFFFFF8D
:10038000FFFFFFFFFFFFFFFFFFFFFFFFFFFFFFFF7D
:10039000FFFFFFFFFFFFFFFFFFFFFFFFFFFFFFFF6D
:1003A000FFFFFFFFFFFFFFFFFFFFFFFFFFFFFFFF5D
:1003B000FFFFFFFFFFFFFFFFFFFFFFFFFFFFFFFF4D
:1003C000FFFFFFFFFFFFFFFFFFFFFFFFFFFFFFFF3D
:1003D000FFFFFFFFFFFFFFFFFFFFFFFFFFFFFFFF2D
:1003E000FFFFFFFFFFFFFFFFFFFFFFFFFFFFFFFF1D
:1003F000FFFFFFFFFFFFFFFFFFFFFFFFFFFFFFFF0D
:020000040030CA
:0E0000000033193C009D84000FC00FE00F403C
:020000040020DA
:08000000FFFFFFFFFFFFFFFF00
:00000001FF
